******************************************************************************
                  TI ARM Linker PC v5.2.2                      
******************************************************************************
>> Linked Sun Sep 20 17:08:06 2015

OUTPUT FILE NAME:   <GPMC_FPGA.out>
ENTRY POINT SYMBOL: "_c_int00"  address: 80009988


MEMORY CONFIGURATION

         name            origin    length      used     unused   attr    fill
----------------------  --------  ---------  --------  --------  ----  --------
  SRAM_LO               402f0000   00000400  00000000  00000400  RW X
  SRAM_HI               402f0400   0000fc00  00000000  0000fc00  RW X
  OCMC_SRAM             40300000   00010000  00000000  00010000  RW X
  DDR3                  80000000   04000000  000189f0  03fe7610  RWIX


SEGMENT ALLOCATION MAP

run origin  load origin   length   init length attrs members
----------  ----------- ---------- ----------- ----- -------
80000000    80000000    0000b808   0000b808    r-x
  80000000    80000000    0000805a   0000805a    r-x .text.1
  8000805c    8000805c    000037a8   000037a8    r-x .text.2
  8000b804    8000b804    00000004   00000004    r-- .const.1
8000b808    8000b808    00004128   00000000    rw-
  8000b808    8000b808    00004128   00000000    rw- .bss
8000f930    8000f930    000006c4   000006c4    r--
  8000f930    8000f930    000006c4   000006c4    r-- .const.2
8000fff4    8000fff4    0000000c   00000000    rw-
  8000fff4    8000fff4    0000000c   00000000    rw- .data.1
80010000    80010000    00004000   00000000    rw-
  80010000    80010000    00004000   00000000    rw- ti.sysbios.family.arm.a8.mmuTableSection
80014000    80014000    0000194e   0000194e    r--
  80014000    80014000    0000194e   0000194e    r-- .const.3
80015950    80015950    0000293c   00000000    rw-
  80015950    80015950    00002000   00000000    rw- .stack
  80017950    80017950    0000093c   00000000    rw- .data.2
80018400    80018400    00000768   00000768    r--
  80018400    80018400    00000040   00000040    r-- .vecs
  80018440    80018440    00000728   00000728    r-- .cinit


SECTION ALLOCATION MAP

 output                                  attributes/
section   page    origin      length       input sections
--------  ----  ----------  ----------   ----------------
.bss       0    8000b808    00004128     UNINITIALIZED
                  8000b808    00002000     app_pea8fnv.oea8fnv (.bss:ti_sysbios_family_arm_exc_Exception_Module_State_0_excStack_0__A)
                  8000d808    00001000     app_pea8fnv.oea8fnv (.bss:ti_sysbios_heaps_HeapMem_Instance_State_0_buf__A)
                  8000e808    00000800     app_pea8fnv.oea8fnv (.bss:taskStackSection)
                  8000f008    00000400     app_pea8fnv.oea8fnv (.bss:ti_sysbios_family_arm_a8_intcps_Hwi_Module_State_0_fiqStack__A)
                  8000f408    00000200     app_pea8fnv.oea8fnv (.bss:xdc_runtime_LoggerBuf_Instance_State_0_entryArr__A)
                  8000f608    00000200     app_pea8fnv.oea8fnv (.bss:xdc_runtime_SysMin_Module_State_0_outbuf__A)
                  8000f808    00000120     rtsv7A8_A_le_n_v3_eabi.lib : trgmsg.obj (.bss:__CIOBUF_)
                  8000f928    00000008     (.common:parmbuf)

.neardata 
*          0    8000f930    00000000     UNINITIALIZED

.rodata    0    8000f930    00000000     UNINITIALIZED

ti.sysbios.family.arm.a8.mmuTableSection 
*          0    80010000    00004000     UNINITIALIZED
                  80010000    00004000     app_pea8fnv.oea8fnv (ti.sysbios.family.arm.a8.mmuTableSection)

.stack     0    80015950    00002000     UNINITIALIZED
                  80015950    00002000     --HOLE--

.cinit     0    80018440    00000728     
                  80018440    000006e5     (.cinit..data.2.load) [load image, compression = rle]
                  80018b25    00000003     --HOLE-- [fill = 0]
                  80018b28    00000011     (.cinit..data.1.load) [load image, compression = rle]
                  80018b39    00000003     --HOLE-- [fill = 0]
                  80018b3c    0000000c     (__TI_handler_table)
                  80018b48    00000008     (.cinit..bss.load) [load image, compression = zero_init]
                  80018b50    00000018     (__TI_cinit_table)

.init_array 
*          0    80000000    00000000     UNINITIALIZED

.text.1    0    80000000    0000805a     
                  80000000    00001c8c     gpmc.obj (.text)
                  80001c8c    000007dc     gpmc_fpga.obj (.text)
                  80002468    00000534     ti.targets.arm.rtsarm.aea8fnv : System.oea8fnv (.text:xdc_runtime_System_doPrint__I)
                  8000299c    000004cc     rtsv7A8_A_le_n_v3_eabi.lib : trgdrv.obj (.text)
                  80002e68    000004cc     sysbios.aea8fnv : BIOS.obj (.text:ti_sysbios_knl_Semaphore_pend__E)
                  80003334    00000390                     : BIOS.obj (.text:ti_sysbios_heaps_HeapMem_free__E)
                  800036c4    0000037c                     : BIOS.obj (.text:ti_sysbios_heaps_HeapMem_alloc__E)
                  80003a40    00000378                     : BIOS.obj (.text:ti_sysbios_knl_Task_Instance_finalize__E)
                  80003db8    00000344     app_pea8fnv.oea8fnv (.text:ti_sysbios_family_arm_a8_Mmu_initTableBuf__I)
                  800040fc    00000324     sysbios.aea8fnv : BIOS.obj (.text:ti_sysbios_knl_Task_sleep__E)
                  80004420    000002fc                     : BIOS.obj (.text:ti_sysbios_family_arm_exc_Exception_excDumpContext__I)
                  8000471c    000002c0                     : BIOS.obj (.text:ti_sysbios_knl_Task_Instance_init__E)
                  800049dc    000002b8     rtsv7A8_A_le_n_v3_eabi.lib : ull_div32.obj (.text)
                  80004c94    0000028c     sysbios.aea8fnv : BIOS.obj (.text:ti_sysbios_family_arm_a8_Mmu_setFirstLevelDesc__E)
                  80004f20    00000280                     : BIOS.obj (.text:ti_sysbios_family_arm_exc_Exception_excHandler__I)
                  800051a0    00000260                     : BIOS.obj (.text:ti_sysbios_knl_Task_Module_startup__E)
                  80005400    00000238     main.obj (.text)
                  80005638    00000228     sysbios.aea8fnv : BIOS.obj (.text:ti_sysbios_timers_dmtimer_Timer_checkFreq__I)
                  80005860    000001fc                     : BIOS.obj (.text:ti_sysbios_family_arm_a8_intcps_Hwi_dispatchIRQC__I)
                  80005a5c    000001f8                     : BIOS.obj (.text:ti_sysbios_heaps_HeapMem_Instance_init__E)
                  80005c54    000001e4                     : BIOS.obj (.text:ti_sysbios_knl_Semaphore_post__E)
                  80005e38    000001d8     ti.targets.arm.rtsarm.aea8fnv : LoggerBuf.oea8fnv (.text:xdc_runtime_LoggerBuf_write8__E)
                  80006010    000001b8     sysbios.aea8fnv : BIOS.obj (.text:ti_sysbios_knl_Clock_workFunc__E)
                  800061c8    000001b0                     : BIOS.obj (.text:ti_sysbios_knl_Swi_run__I)
                  80006378    000001b0                     : BIOS.obj (.text:ti_sysbios_timers_dmtimer_Timer_deviceConfig__I)
                  80006528    000001a8     ti.targets.arm.rtsarm.aea8fnv : Error.oea8fnv (.text:xdc_runtime_Error_policyDefault__E)
                  800066d0    000001a4                                   : Core-mem.oea8fnv (.text:xdc_runtime_Core_createObject__I)
                  80006874    00000188     app_pea8fnv.oea8fnv (.text:xdc_runtime_System_printfExtend__I)
                  800069fc    00000180     rtsv7A8_A_le_n_v3_eabi.lib : memcpy32.obj (.text)
                  80006b7c    00000178     sysbios.aea8fnv : BIOS.obj (.text:ti_sysbios_family_arm_a8_Cache_startup__I)
                  80006cf4    0000015c                     : BIOS.obj (.text:ti_sysbios_family_arm_a8_intcps_Hwi_Module_startup__E)
                  80006e50    00000154     ti.targets.arm.rtsarm.aea8fnv : Startup.oea8fnv (.text:xdc_runtime_Startup_startMods__I)
                  80006fa4    00000144                                   : Core-smem.oea8fnv (.text:xdc_runtime_Core_constructObject__I)
                  800070e8    0000013c     sysbios.aea8fnv : BIOS.obj (.text:ti_sysbios_knl_Task_schedule__I)
                  80007224    0000013c                     : BIOS.obj (.text:ti_sysbios_knl_Task_startCore__E)
                  80007360    0000013c                     : BIOS.obj (.text:ti_sysbios_timers_dmtimer_Timer_setPeriodMicroSecs__E)
                  8000749c    00000134                     : BIOS.obj (.text:ti_sysbios_knl_Task_checkStacks__E)
                  800075d0    00000134     ti.targets.arm.rtsarm.aea8fnv : LoggerBuf.oea8fnv (.text:xdc_runtime_LoggerBuf_write4__E)
                  80007704    00000124     sysbios.aea8fnv : BIOS.obj (.text:ti_sysbios_family_arm_a8_Mmu_initDescAttrs__E)
                  80007828    00000124                     : BIOS.obj (.text:ti_sysbios_gates_GateMutex_enter__E)
                  8000794c    00000124                     : BIOS.obj (.text:ti_sysbios_knl_Swi_post__E)
                  80007a70    00000108                     : BIOS.obj (.text:ti_sysbios_knl_Semaphore_Instance_init__E)
                  80007b78    00000104                     : BIOS.obj (.text:ti_sysbios_knl_Task_postInit__I)
                  80007c7c    000000fc                     : BIOS.obj (.text:ti_sysbios_knl_Task_blockI__E)
                  80007d78    000000fc                     : BIOS.obj (.text:ti_sysbios_knl_Task_unblockI__E)
                  80007e74    000000f4     rtsv7A8_A_le_n_v3_eabi.lib : u_div32.obj (.text)
                  80007f68    000000f2     ti.targets.arm.rtsarm.aea8fnv : Text.oea8fnv (.text:xdc_runtime_Text_putSite__E)

.text.2    0    8000805c    000037a8     
                  8000805c    000000f0     sysbios.aea8fnv : BIOS.obj (.text:ti_sysbios_family_arm_a8_intcps_Hwi_disableInterrupt__E)
                  8000814c    000000f0                     : BIOS.obj (.text:ti_sysbios_family_arm_a8_intcps_Hwi_enableInterrupt__E)
                  8000823c    000000ec     auto_init.aea8fnv : auto_init.oea8fnv (.text)
                  80008328    000000ec     sysbios.aea8fnv : BIOS.obj (.text:ti_sysbios_knl_Task_exit__E)
                  80008414    000000dc                     : BIOS.obj (.text:ti_sysbios_timers_dmtimer_Timer_start__E)
                  800084f0    000000d8     ti.targets.arm.rtsarm.aea8fnv : LoggerBuf.oea8fnv (.text:xdc_runtime_LoggerBuf_setFilterLevel__E)
                  800085c8    000000d8                                   : Text.oea8fnv (.text:xdc_runtime_Text_putMod__E)
                  800086a0    000000d0     sysbios.aea8fnv : exc_Exception_asm.obj (.text:ti_sysbios_family_arm_exc_Exception_excHandlerAsm__I)
                  80008770    000000cc     ti.targets.arm.rtsarm.aea8fnv : LoggerBuf.oea8fnv (.text:xdc_runtime_LoggerBuf_getFilterLevel__E)
                  8000883c    000000c0     sysbios.aea8fnv : intcps_Hwi_asm.obj (.text:ti_sysbios_family_arm_a8_intcps_Hwi_dispatchIRQ__I)
                  800088fc    000000b4                     : BIOS.obj (.text:ti_sysbios_timers_dmtimer_Timer_Module_startup__E)
                  800089b0    000000b0     rtsv7A8_A_le_n_v3_eabi.lib : memset32.obj (.text)
                  80008a60    000000b0     ti.targets.arm.rtsarm.aea8fnv : Memory.oea8fnv (.text:xdc_runtime_Memory_alloc__E)
                  80008b10    000000a4     rtsv7A8_A_le_n_v3_eabi.lib : trgmsg.obj (.text)
                  80008bb4    000000a0                                : copy_decompress_rle.obj (.text)
                  80008c54    0000009f     ti.targets.arm.rtsarm.aea8fnv : Text.oea8fnv (.text:xdc_runtime_Text_putLab__E)
                  80008cf3    00000001     --HOLE-- [fill = 0]
                  80008cf4    0000009c     sysbios.aea8fnv : BIOS.obj (.text:ti_sysbios_knl_Clock_logTick__E)
                  80008d90    0000009c                     : BIOS.obj (.text:ti_sysbios_knl_Swi_restoreHwi__E)
                  80008e2c    00000098     app_pea8fnv.oea8fnv (.text:ti_sysbios_knl_Task_create)
                  80008ec4    00000098     ti.targets.arm.rtsarm.aea8fnv : Core-mem.oea8fnv (.text:xdc_runtime_Core_deleteObject__I)
                  80008f5c    00000098                                   : Error.oea8fnv (.text:xdc_runtime_Error_print__E)
                  80008ff4    00000098     app_pea8fnv.oea8fnv (.text:xdc_runtime_LoggerBuf_Object__create__S)
                  8000908c    00000098     ti.targets.arm.rtsarm.aea8fnv : System.oea8fnv (.text:xdc_runtime_System_formatNum__I)
                  80009124    00000094     sysbios.aea8fnv : a8_Cache_asm.obj (.text:ti_sysbios_family_arm_a8_Cache_invL1dAll__E)
                  800091b8    00000094                     : a8_Cache_asm.obj (.text:ti_sysbios_family_arm_a8_Cache_wbInvAll__E)
                  8000924c    00000094                     : BIOS.obj (.text:ti_sysbios_timers_dmtimer_Timer_initDevice__I)
                  800092e0    0000008c                     : intcps_Hwi_asm_switch.obj (.text:_ti_sysbios_family_xxx_Hwi_switchToIsrStack)
                  8000936c    0000008c     sys_bios_driver.lib : osdrv_mmu.obj (.text)
                  800093f8    0000008c     ti.targets.arm.rtsarm.aea8fnv : Startup.oea8fnv (.text:xdc_runtime_Startup_exec__E)
                  80009484    00000088     sysbios.aea8fnv : BIOS.obj (.text:ti_sysbios_family_arm_a8_Mmu_Module_startup__E)
                  8000950c    00000084     rtsv7A8_A_le_n_v3_eabi.lib : cpy_tbl.obj (.text)
                  80009590    00000084     sysbios.aea8fnv : BIOS.obj (.text:ti_sysbios_knl_Swi_schedule__I)
                  80009614    00000084                     : BIOS.obj (.text:ti_sysbios_knl_Task_allBlockedFunction__I)
                  80009698    00000080                     : BIOS.obj (.text:ti_sysbios_heaps_HeapMem_getStats__E)
                  80009718    00000080                     : BIOS.obj (.text:ti_sysbios_knl_Swi_runLoop__I)
                  80009798    00000080     ti.targets.arm.rtsarm.aea8fnv : Text.oea8fnv (.text:xdc_runtime_Text_visitRope2__I)
                  80009818    0000007c     sysbios.aea8fnv : arm_TaskSupport_asm.obj (.text:_ti_sysbios_family_arm_TaskSupport_buildTaskStack)
                  80009894    0000007c     ti.targets.arm.rtsarm.aea8fnv : Assert.oea8fnv (.text:xdc_runtime_Assert_raise__I)
                  80009910    00000078     rtsv7A8_A_le_n_v3_eabi.lib : exit.obj (.text)
                  80009988    00000074     boot.aea8fnv : boot.oea8fnv (.text)
                  800099fc    00000074     sysbios.aea8fnv : BIOS.obj (.text:ti_sysbios_family_arm_a8_intcps_Hwi_dispatchFIQC__I)
                  80009a70    00000074                     : BIOS.obj (.text:ti_sysbios_timers_dmtimer_Timer_startup__E)
                  80009ae4    00000074     ti.targets.arm.rtsarm.aea8fnv : LoggerBuf.oea8fnv (.text:xdc_runtime_LoggerBuf_filterOutEvent__I)
                  80009b58    00000070     sysbios.aea8fnv : BIOS.obj (.text:ti_sysbios_family_arm_a8_Mmu_enable__E)
                  80009bc8    00000070     ti.targets.arm.rtsarm.aea8fnv : SysMin.oea8fnv (.text:xdc_runtime_SysMin_flush__E)
                  80009c38    0000006c     sysbios.aea8fnv : BIOS.obj (.text:ti_sysbios_family_arm_a8_intcps_Hwi_getStackInfo__E)
                  80009ca4    00000068                     : BIOS.obj (.text:ti_sysbios_family_arm_TaskSupport_start__E)
                  80009d0c    00000068                     : BIOS.obj (.text:ti_sysbios_heaps_HeapMem_init__I)
                  80009d74    00000068     ti.targets.arm.rtsarm.aea8fnv : Error.oea8fnv (.text:xdc_runtime_Error_setX__E)
                  80009ddc    00000068                                   : LoggerBuf.oea8fnv (.text:xdc_runtime_LoggerBuf_Instance_init__E)
                  80009e44    00000064     sysbios.aea8fnv : BIOS.obj (.text:ti_sysbios_family_arm_a8_Cache_disable__E)
                  80009ea8    00000064                     : exc_Exception_asm.obj (.text:ti_sysbios_family_arm_exc_Exception_initCore0__I)
                  80009f0c    00000064     ti.targets.arm.rtsarm.aea8fnv : Core-params.oea8fnv (.text:xdc_runtime_Core_assignParams__I)
                  80009f70    00000060     sysbios.aea8fnv : BIOS.obj (.text:ti_sysbios_timers_dmtimer_Timer_stop__E)
                  80009fd0    00000060     ti.targets.arm.rtsarm.aea8fnv : Text.oea8fnv (.text:xdc_runtime_Text_xprintf__I)
                  8000a030    0000005c     sysbios.aea8fnv : BIOS.obj (.text:ti_sysbios_knl_Task_restore__E)
                  8000a08c    0000005c     ti.targets.arm.rtsarm.aea8fnv : Core-label.oea8fnv (.text:xdc_runtime_Core_assignLabel__I)
                  8000a0e8    0000005c                                   : SysMin.oea8fnv (.text:xdc_runtime_SysMin_putch__E)
                  8000a144    0000005c                                   : System.oea8fnv (.text:xdc_runtime_System_atexit__E)
                  8000a1a0    00000058     sysbios.aea8fnv : BIOS.obj (.text:ti_sysbios_family_arm_a8_intcps_Hwi_nonPluggedHwiHandler__I)
                  8000a1f8    00000058                     : BIOS.obj (.text:ti_sysbios_hal_Hwi_checkStack)
                  8000a250    00000058                     : BIOS.obj (.text:ti_sysbios_knl_Swi_startup__E)
                  8000a2a8    00000058     ti.targets.arm.rtsarm.aea8fnv : SysMin.oea8fnv (.text:xdc_runtime_SysMin_abort__E)
                  8000a300    00000054     sysbios.aea8fnv : BIOS.obj (.text:ti_sysbios_knl_Semaphore_pendTimeout__I)
                  8000a354    00000054                     : BIOS.obj (.text:ti_sysbios_knl_Task_processVitalTaskFlag__I)
                  8000a3a8    00000054     ti.targets.arm.rtsarm.aea8fnv : System.oea8fnv (.text:xdc_runtime_System_putchar__I)
                  8000a3fc    00000053                                   : Text.oea8fnv (.text:xdc_runtime_Text_printVisFxn__I)
                  8000a44f    00000001     --HOLE-- [fill = 0]
                  8000a450    00000050     app_pea8fnv.oea8fnv (.text:ti_sysbios_gates_GateHwi_Object__create__S)
                  8000a4a0    00000050     app_pea8fnv.oea8fnv (.text:ti_sysbios_gates_GateMutex_Object__create__S)
                  8000a4f0    00000050     app_pea8fnv.oea8fnv (.text:ti_sysbios_heaps_HeapMem_Object__create__S)
                  8000a540    00000050     app_pea8fnv.oea8fnv (.text:ti_sysbios_knl_Semaphore_construct)
                  8000a590    0000004c     sysbios.aea8fnv : BIOS.obj (.text:ti_sysbios_family_arm_a8_TimestampProvider_get64__E)
                  8000a5dc    0000004c                     : BIOS.obj (.text:ti_sysbios_hal_Hwi_initStack)
                  8000a628    00000048     app_pea8fnv.oea8fnv (.text:ti_sysbios_knl_Queue_construct)
                  8000a670    00000048     ti.targets.arm.rtsarm.aea8fnv : System.oea8fnv (.text:xdc_runtime_System_processAtExit__E)
                  8000a6b8    00000044     app_pea8fnv.oea8fnv (.text:ti_sysbios_BIOS_atExitFunc__I)
                  8000a6fc    00000044     app_pea8fnv.oea8fnv (.text:ti_sysbios_knl_Clock_doTick__I)
                  8000a740    00000044     sysbios.aea8fnv : BIOS.obj (.text:ti_sysbios_knl_Task_restoreHwi__E)
                  8000a784    00000044     app_pea8fnv.oea8fnv (.text:xdc_runtime_SysMin_output__I)
                  8000a7c8    00000044     ti.targets.arm.rtsarm.aea8fnv : Text.oea8fnv (.text:xdc_runtime_Text_cordText__E)
                  8000a80c    00000040     am335x_platform.lib : plat_mux.obj (.text)
                  8000a84c    00000040     sysbios.aea8fnv : BIOS.obj (.text:ti_sysbios_family_arm_a8_Cache_enable__E)
                  8000a88c    00000040     ti.targets.arm.rtsarm.aea8fnv : LoggerBuf.oea8fnv (.text:xdc_runtime_LoggerBuf_Module_startup__E)
                  8000a8cc    00000040                                   : System.oea8fnv (.text:xdc_runtime_System_avprintf__E)
                  8000a90c    0000003c     sysbios.aea8fnv : BIOS.obj (.text:ti_sysbios_family_arm_a8_Mmu_disable__E)
                  8000a948    0000003c                     : BIOS.obj (.text:ti_sysbios_family_arm_a8_TimestampProvider_autoRefreshFxn__I)
                  8000a984    0000003c                     : BIOS.obj (.text:ti_sysbios_knl_Swi_Module_startup__E)
                  8000a9c0    0000003c                     : BIOS.obj (.text:ti_sysbios_timers_dmtimer_Timer_stub__E)
                  8000a9fc    0000003c     ti.targets.arm.rtsarm.aea8fnv : System.oea8fnv (.text:xdc_runtime_System_vprintf__E)
                  8000aa38    00000038     sysbios.aea8fnv : a8_Cache_asm.obj (.text:ti_sysbios_family_arm_a8_Cache_getEnabled__E)
                  8000aa70    00000038     ti.targets.arm.rtsarm.aea8fnv : LoggerBuf.oea8fnv (.text:xdc_runtime_LoggerBuf_reset__E)
                  8000aaa8    00000034     app_pea8fnv.oea8fnv (.text:ti_sysbios_BIOS_errorRaiseHook__I)
                  8000aadc    00000034     app_pea8fnv.oea8fnv (.text:ti_sysbios_BIOS_registerRTSLock__I)
                  8000ab10    00000034     app_pea8fnv.oea8fnv (.text:ti_sysbios_BIOS_removeRTSLock__I)
                  8000ab44    00000034     app_pea8fnv.oea8fnv (.text:ti_sysbios_gates_GateMutex_Object__delete__S)
                  8000ab78    00000034     sysbios.aea8fnv : BIOS.obj (.text:ti_sysbios_knl_Clock_Module_startup__E)
                  8000abac    00000034                     : BIOS.obj (.text:ti_sysbios_knl_Idle_run__E)
                  8000abe0    00000034                     : BIOS.obj (.text:ti_sysbios_knl_Task_enter__I)
                  8000ac14    00000034     app_pea8fnv.oea8fnv (.text:xdc_runtime_LoggerBuf_Object__delete__S)
                  8000ac48    00000034     ti.targets.arm.rtsarm.aea8fnv : Registry.oea8fnv (.text:xdc_runtime_Registry_findById__E)
                  8000ac7c    00000034                                   : SysMin.oea8fnv (.text:xdc_runtime_SysMin_Module_startup__E)
                  8000acb0    00000030     sysbios.aea8fnv : a8_Mmu_asm.obj (.text:_ti_sysbios_family_arm_a8_Mmu_enableAsm)
                  8000ace0    00000030     app_pea8fnv.oea8fnv (.text:ti_sysbios_BIOS_rtsLock__I)
                  8000ad10    00000030     app_pea8fnv.oea8fnv (.text:ti_sysbios_gates_GateHwi_Object__delete__S)
                  8000ad40    00000030     sysbios.aea8fnv : BIOS.obj (.text:ti_sysbios_gates_GateMutex_Instance_init__E)
                  8000ad70    00000030     app_pea8fnv.oea8fnv (.text:ti_sysbios_heaps_HeapMem_Object__delete__S)
                  8000ada0    00000030     ti.targets.arm.rtsarm.aea8fnv : Error.oea8fnv (.text:xdc_runtime_Error_raiseX__E)
                  8000add0    00000030                                   : Memory.oea8fnv (.text:xdc_runtime_Memory_valloc__E)
                  8000ae00    00000030                                   : SysMin.oea8fnv (.text:xdc_runtime_SysMin_exit__E)
                  8000ae30    0000002c     app_pea8fnv.oea8fnv (.text:ti_sysbios_gates_GateHwi_Handle__label__S)
                  8000ae5c    0000002c     app_pea8fnv.oea8fnv (.text:ti_sysbios_gates_GateMutex_Handle__label__S)
                  8000ae88    0000002c     sysbios.aea8fnv : BIOS.obj (.text:ti_sysbios_gates_GateMutex_leave__E)
                  8000aeb4    0000002c     app_pea8fnv.oea8fnv (.text:ti_sysbios_heaps_HeapMem_Handle__label__S)
                  8000aee0    0000002c     app_pea8fnv.oea8fnv (.text:ti_sysbios_knl_Semaphore_Object__destruct__S)
                  8000af0c    0000002c     ti.targets.arm.rtsarm.aea8fnv : Error.oea8fnv (.text:xdc_runtime_Error_check__E)
                  8000af38    0000002c     app_pea8fnv.oea8fnv (.text:xdc_runtime_LoggerBuf_Handle__label__S)
                  8000af64    00000028     app_pea8fnv.oea8fnv (.text:ti_sysbios_BIOS_rtsUnlock__I)
                  8000af8c    00000028     app_pea8fnv.oea8fnv (.text:ti_sysbios_BIOS_startFunc__I)
                  8000afb4    00000028     app_pea8fnv.oea8fnv (.text:ti_sysbios_family_arm_a8_intcps_Hwi_Module__startupDone__F)
                  8000afdc    00000028     app_pea8fnv.oea8fnv (.text:ti_sysbios_family_arm_a8_ti81xx_TimerSupport_Module__startupDone__F)
                  8000b004    00000028     app_pea8fnv.oea8fnv (.text:ti_sysbios_knl_Queue_Object__destruct__S)
                  8000b02c    00000028     app_pea8fnv.oea8fnv (.text:ti_sysbios_timers_dmtimer_Timer_Module__startupDone__F)
                  8000b054    00000028     ti.targets.arm.rtsarm.aea8fnv : System.oea8fnv (.text:xdc_runtime_System_abort__E)
                  8000b07c    00000028     app_pea8fnv.oea8fnv (.text:xdc_runtime_System_aprintf__E)
                  8000b0a4    00000028     app_pea8fnv.oea8fnv (.text:xdc_runtime_System_printf__E)
                  8000b0cc    00000024     rtsv7A8_A_le_n_v3_eabi.lib : _lock.obj (.text)
                  8000b0f0    00000024     sysbios.aea8fnv : intcps_Hwi_asm.obj (.text:ti_sysbios_family_arm_a8_intcps_Hwi_init__I)
                  8000b114    00000024                     : BIOS.obj (.text:ti_sysbios_knl_Task_sleepTimeout__I)
                  8000b138    00000024     ti.targets.arm.rtsarm.aea8fnv : System.oea8fnv (.text:xdc_runtime_System_exit__E)
                  8000b15c    00000020     sysbios.aea8fnv : a8_Mmu_asm.obj (.text:_ti_sysbios_family_arm_a8_Mmu_disableAsm)
                  8000b17c    00000020     rtsv7A8_A_le_n_v3_eabi.lib : args_main.obj (.text)
                  8000b19c    00000020     app_pea8fnv.oea8fnv (.text:ti_sysbios_BIOS_exitFunc__I)
                  8000b1bc    00000020     sysbios.aea8fnv : BIOS.obj (.text:ti_sysbios_family_arm_a8_intcps_Hwi_startup__E)
                  8000b1dc    00000020     ti.targets.arm.rtsarm.aea8fnv : LoggerBuf.oea8fnv (.text:xdc_runtime_LoggerBuf_Instance_finalize__E)
                  8000b1fc    00000020                                   : LoggerBuf.oea8fnv (.text:xdc_runtime_LoggerBuf_write2__E)
                  8000b21c    0000001c     sysbios.aea8fnv : arm_TaskSupport_asm.obj (.text:_ti_sysbios_family_arm_TaskSupport_glue)
                  8000b238    0000001c     rtsv7A8_A_le_n_v3_eabi.lib : strlen.obj (.text)
                  8000b254    0000001c     sysbios.aea8fnv : a8_Cache_asm.obj (.text:ti_sysbios_family_arm_a8_Cache_disableBP__E)
                  8000b270    0000001c                     : a8_Cache_asm.obj (.text:ti_sysbios_family_arm_a8_Cache_disableL1d__I)
                  8000b28c    0000001c                     : a8_Cache_asm.obj (.text:ti_sysbios_family_arm_a8_Cache_enableBP__E)
                  8000b2a8    0000001c                     : a8_TimestampProvider_asm.obj (.text:ti_sysbios_family_arm_a8_TimestampProvider_initCCNT__I)
                  8000b2c4    0000001c     app_pea8fnv.oea8fnv (.text:ti_sysbios_heaps_HeapMem_Object__get__S)
                  8000b2e0    0000001c     app_pea8fnv.oea8fnv (.text:ti_sysbios_knl_Swi_Object__get__S)
                  8000b2fc    0000001c     app_pea8fnv.oea8fnv (.text:xdc_runtime_LoggerBuf_Object__get__S)
                  8000b318    0000001c     ti.targets.arm.rtsarm.aea8fnv : LoggerBuf.oea8fnv (.text:xdc_runtime_LoggerBuf_write0__E)
                  8000b334    0000001c                                   : LoggerBuf.oea8fnv (.text:xdc_runtime_LoggerBuf_write1__E)
                  8000b350    0000001c     app_pea8fnv.oea8fnv (.text:xdc_runtime_Startup_exec__I)
                  8000b36c    0000001c     ti.targets.arm.rtsarm.aea8fnv : SysMin.oea8fnv (.text:xdc_runtime_SysMin_ready__E)
                  8000b388    0000001c                                   : System.oea8fnv (.text:xdc_runtime_System_vsnprintf__E)
                  8000b3a4    0000001c                                   : Text.oea8fnv (.text:xdc_runtime_Text_ropeText__E)
                  8000b3c0    00000018     sysbios.aea8fnv : arm_TaskSupport_asm.obj (.text:_ti_sysbios_family_arm_TaskSupport_swap__E)
                  8000b3d8    00000018     rtsv7A8_A_le_n_v3_eabi.lib : strcpy.obj (.text)
                  8000b3f0    00000018     sysbios.aea8fnv : BIOS.obj (.text:ti_sysbios_BIOS_exit__E)
                  8000b408    00000018                     : BIOS.obj (.text:ti_sysbios_BIOS_setThreadType__E)
                  8000b420    00000018                     : BIOS.obj (.text:ti_sysbios_BIOS_start__E)
                  8000b438    00000018                     : BIOS.obj (.text:ti_sysbios_hal_Hwi_Module_startup__E)
                  8000b450    00000018                     : BIOS.obj (.text:ti_sysbios_knl_Queue_empty__E)
                  8000b468    00000018                     : BIOS.obj (.text:ti_sysbios_knl_Swi_disable__E)
                  8000b480    00000018     app_pea8fnv.oea8fnv (.text:ti_sysbios_knl_Task_Object__get__S)
                  8000b498    00000018     sysbios.aea8fnv : BIOS.obj (.text:ti_sysbios_knl_Task_disable__E)
                  8000b4b0    00000018     ti.targets.arm.rtsarm.aea8fnv : Error.oea8fnv (.text:xdc_runtime_Error_init__E)
                  8000b4c8    00000018     app_pea8fnv.oea8fnv (.text:xdc_runtime_Text_visitRope__I)
                  8000b4e0    00000014     sysbios.aea8fnv : a8_Mmu_asm.obj (.text:_ti_sysbios_family_arm_a8_Mmu_init)
                  8000b4f4    00000014                     : a8_Mmu_asm.obj (.text:_ti_sysbios_family_arm_a8_Mmu_isEnabled)
                  8000b508    00000014     rtsv7A8_A_le_n_v3_eabi.lib : copy_decompress_none.obj (.text:decompress:none)
                  8000b51c    00000014     sysbios.aea8fnv : BIOS.obj (.text:ti_sysbios_family_arm_TaskSupport_checkStack__E)
                  8000b530    00000014                     : a8_Cache_asm.obj (.text:ti_sysbios_family_arm_a8_Cache_disableL1p__I)
                  8000b544    00000014                     : a8_Cache_asm.obj (.text:ti_sysbios_family_arm_a8_Cache_enableL1p__I)
                  8000b558    00000014                     : BIOS.obj (.text:ti_sysbios_family_arm_a8_intcps_Hwi_clearInterrupt__E)
                  8000b56c    00000014                     : BIOS.obj (.text:ti_sysbios_family_arm_a8_intcps_Hwi_switchFromBootStack__E)
                  8000b580    00000014                     : BIOS.obj (.text:ti_sysbios_gates_GateMutex_Instance_finalize__E)
                  8000b594    00000014                     : BIOS.obj (.text:ti_sysbios_knl_Semaphore_Instance_finalize__E)
                  8000b5a8    00000014     ti.targets.arm.rtsarm.aea8fnv : Gate.oea8fnv (.text:xdc_runtime_Gate_leaveSystem__E)
                  8000b5bc    00000014     app_pea8fnv.oea8fnv (.text:xdc_runtime_IHeap_alloc)
                  8000b5d0    00000014     app_pea8fnv.oea8fnv (.text:xdc_runtime_IHeap_free)
                  8000b5e4    00000014     ti.targets.arm.rtsarm.aea8fnv : LoggerBuf.oea8fnv (.text:xdc_runtime_LoggerBuf_disable__E)
                  8000b5f8    00000014                                   : LoggerBuf.oea8fnv (.text:xdc_runtime_LoggerBuf_enable__E)
                  8000b60c    00000014                                   : Memory.oea8fnv (.text:xdc_runtime_Memory_calloc__E)
                  8000b620    00000014                                   : Memory.oea8fnv (.text:xdc_runtime_Memory_free__E)
                  8000b634    00000010     rtsv7A8_A_le_n_v3_eabi.lib : copy_zero_init.obj (.text:decompress:ZI)
                  8000b644    00000010     sysbios.aea8fnv : BIOS.obj (.text:ti_sysbios_BIOS_getCpuFreq__E)
                  8000b654    00000010                     : BIOS.obj (.text:ti_sysbios_family_arm_TaskSupport_getStackAlignment__E)
                  8000b664    00000010                     : a8_Cache_asm.obj (.text:ti_sysbios_family_arm_a8_Cache_disableL2__I)
                  8000b674    00000010                     : a8_Cache_asm.obj (.text:ti_sysbios_family_arm_a8_Cache_enableL1d__I)
                  8000b684    00000010                     : a8_Cache_asm.obj (.text:ti_sysbios_family_arm_a8_Cache_enableL2__I)
                  8000b694    00000010                     : BIOS.obj (.text:ti_sysbios_family_arm_a8_TimestampProvider_Module_startup__E)
                  8000b6a4    00000010                     : intcps_Hwi_asm.obj (.text:ti_sysbios_family_arm_a8_intcps_Hwi_initVbar__I)
                  8000b6b4    00000010                     : BIOS.obj (.text:ti_sysbios_family_arm_exc_Exception_Module_startup__E)
                  8000b6c4    00000010                     : BIOS.obj (.text:ti_sysbios_gates_GateHwi_enter__E)
                  8000b6d4    00000010     app_pea8fnv.oea8fnv (.text:ti_sysbios_knl_Queue_Object__get__S)
                  8000b6e4    00000010     ti.targets.arm.rtsarm.aea8fnv : Gate.oea8fnv (.text:xdc_runtime_Gate_enterSystem__E)
                  8000b6f4    00000010                                   : Memory.oea8fnv (.text:xdc_runtime_Memory_getMaxDefaultTypeAlign__E)
                  8000b704    00000010                                   : Startup.oea8fnv (.text:xdc_runtime_Startup_rtsDone__E)
                  8000b714    0000000c     sysbios.aea8fnv : a8_Cache_asm.obj (.text:ti_sysbios_family_arm_a8_Cache_getCacheLevelInfo__I)
                  8000b720    0000000c                     : BIOS.obj (.text:ti_sysbios_knl_Idle_loop__E)
                  8000b72c    0000000c                     : BIOS.obj (.text:ti_sysbios_knl_Queue_Instance_init__E)
                  8000b738    0000000c                     : BIOS.obj (.text:ti_sysbios_timers_dmtimer_Timer_getMaxTicks__E)
                  8000b744    00000008     ti.targets.arm.rtsarm.aea8fnv : xdc_noinit.oea8fnv (.text:__xdc__init)
                  8000b74c    00000008     sysbios.aea8fnv : a8_Mmu_asm.obj (.text:_ti_sysbios_family_arm_a8_Mmu_setDomainAccessCtrlReg)
                  8000b754    00000008     rtsv7A8_A_le_n_v3_eabi.lib : copy_decompress_rle.obj (.text:decompress:rle24)
                  8000b75c    00000008     app_pea8fnv.oea8fnv (.text:ti_sysbios_family_arm_TaskSupport_Module__startupDone__S)
                  8000b764    00000008     sysbios.aea8fnv : a8_Cache_asm.obj (.text:ti_sysbios_family_arm_a8_Cache_getLockdownReg__I)
                  8000b76c    00000008                     : a8_Cache_asm.obj (.text:ti_sysbios_family_arm_a8_Cache_invL1pAll__E)
                  8000b774    00000008                     : a8_Cache_asm.obj (.text:ti_sysbios_family_arm_a8_Cache_setLockdownReg__I)
                  8000b77c    00000008                     : a8_TimestampProvider_asm.obj (.text:ti_sysbios_family_arm_a8_TimestampProvider_get32__E)
                  8000b784    00000008                     : BIOS.obj (.text:ti_sysbios_family_arm_a8_ti81xx_TimerSupport_Module_startup__E)
                  8000b78c    00000008                     : BIOS.obj (.text:ti_sysbios_gates_GateHwi_leave__E)
                  8000b794    00000008                     : BIOS.obj (.text:ti_sysbios_gates_GateHwi_query__E)
                  8000b79c    00000008                     : BIOS.obj (.text:ti_sysbios_gates_GateMutex_query__E)
                  8000b7a4    00000008                     : BIOS.obj (.text:ti_sysbios_heaps_HeapMem_isBlocking__E)
                  8000b7ac    00000008     ti.targets.arm.rtsarm.aea8fnv : Error.oea8fnv (.text:xdc_runtime_Error_getSite__E)
                  8000b7b4    00000008                                   : System.oea8fnv (.text:xdc_runtime_System_Module_startup__E)
                  8000b7bc    00000004                                   : LoggerBuf.oea8fnv (.text:LoggerBuf_instanceStartup)
                  8000b7c0    00000004     app_pea8fnv.oea8fnv (.text:ti_sysbios_BIOS_RtsGateProxy_enter__E)
                  8000b7c4    00000004     app_pea8fnv.oea8fnv (.text:ti_sysbios_BIOS_RtsGateProxy_leave__E)
                  8000b7c8    00000004     app_pea8fnv.oea8fnv (.text:ti_sysbios_BIOS_nullFunc__I)
                  8000b7cc    00000004     sysbios.aea8fnv : BIOS.obj (.text:ti_sysbios_family_arm_a8_ti81xx_TimerSupport_enable__E)
                  8000b7d0    00000004                     : BIOS.obj (.text:ti_sysbios_gates_GateHwi_Instance_init__E)
                  8000b7d4    00000004     app_pea8fnv.oea8fnv (.text:ti_sysbios_heaps_HeapMem_Module_GateProxy_enter__E)
                  8000b7d8    00000004     app_pea8fnv.oea8fnv (.text:ti_sysbios_heaps_HeapMem_Module_GateProxy_leave__E)
                  8000b7dc    00000004     app_pea8fnv.oea8fnv (.text:ti_sysbios_knl_Clock_TimerProxy_getMaxTicks__E)
                  8000b7e0    00000004     app_pea8fnv.oea8fnv (.text:ti_sysbios_knl_Queue_destruct)
                  8000b7e4    00000004     app_pea8fnv.oea8fnv (.text:ti_sysbios_knl_Semaphore_destruct)
                  8000b7e8    00000004     sysbios.aea8fnv : BIOS.obj (.text:ti_sysbios_knl_Task_startup__E)
                  8000b7ec    00000004     app_pea8fnv.oea8fnv (.text:xdc_runtime_LoggerBuf_Module_GateProxy_enter__E)
                  8000b7f0    00000004     app_pea8fnv.oea8fnv (.text:xdc_runtime_LoggerBuf_Module_GateProxy_leave__E)
                  8000b7f4    00000004     app_pea8fnv.oea8fnv (.text:xdc_runtime_System_Module_GateProxy_enter__E)
                  8000b7f8    00000004     app_pea8fnv.oea8fnv (.text:xdc_runtime_System_Module_GateProxy_leave__E)
                  8000b7fc    00000004     ti.targets.arm.rtsarm.aea8fnv : System.oea8fnv (.text:xdc_runtime_System_aprintf_va__F)
                  8000b800    00000004                                   : System.oea8fnv (.text:xdc_runtime_System_printf_va__F)

.const.1   0    8000b804    00000004     
                  8000b804    00000004     app_pea8fnv.oea8fnv (.const:ti_sysbios_family_arm_TaskSupport_stackAlignment__C)

.const.2   0    8000f930    000006c4     
                  8000f930    000000e0     app_pea8fnv.oea8fnv (.const:xdc_runtime_Text_nodeTab__A)
                  8000fa10    00000048     app_pea8fnv.oea8fnv (.const:.string)
                  8000fa58    0000003c     app_pea8fnv.oea8fnv (.const:ti_sysbios_knl_Task_Object__PARAMS__C)
                  8000fa94    0000003c     app_pea8fnv.oea8fnv (.const:xdc_runtime_LoggerBuf_Module__FXNS__C)
                  8000fad0    00000034     app_pea8fnv.oea8fnv (.const:xdc_runtime_Startup_sfxnTab__A)
                  8000fb04    00000028     app_pea8fnv.oea8fnv (.const:ti_sysbios_heaps_HeapMem_Module__FXNS__C)
                  8000fb2c    00000024     app_pea8fnv.oea8fnv (.const:ti_sysbios_gates_GateHwi_Module__FXNS__C)
                  8000fb50    00000024     app_pea8fnv.oea8fnv (.const:ti_sysbios_gates_GateMutex_Module__FXNS__C)
                  8000fb74    00000024     app_pea8fnv.oea8fnv (.const:ti_sysbios_heaps_HeapMem_Object__PARAMS__C)
                  8000fb98    00000024     app_pea8fnv.oea8fnv (.const:ti_sysbios_knl_Semaphore_Object__PARAMS__C)
                  8000fbbc    00000024     app_pea8fnv.oea8fnv (.const:xdc_runtime_LoggerBuf_Object__PARAMS__C)
                  8000fbe0    00000020     app_pea8fnv.oea8fnv (.const:ti_sysbios_gates_GateHwi_Object__DESC__C)
                  8000fc00    00000020     app_pea8fnv.oea8fnv (.const:ti_sysbios_gates_GateMutex_Object__DESC__C)
                  8000fc20    00000020     app_pea8fnv.oea8fnv (.const:ti_sysbios_heaps_HeapMem_Object__DESC__C)
                  8000fc40    00000020     app_pea8fnv.oea8fnv (.const:ti_sysbios_knl_Queue_Object__DESC__C)
                  8000fc60    00000020     app_pea8fnv.oea8fnv (.const:ti_sysbios_knl_Semaphore_Object__DESC__C)
                  8000fc80    00000020     app_pea8fnv.oea8fnv (.const:ti_sysbios_knl_Task_Object__DESC__C)
                  8000fca0    00000020     app_pea8fnv.oea8fnv (.const:xdc_runtime_LoggerBuf_Object__DESC__C)
                  8000fcc0    0000001a     app_pea8fnv.oea8fnv (.const:xdc_runtime_Startup_sfxnRts__A)
                  8000fcda    00000002     app_pea8fnv.oea8fnv (.const:ti_sysbios_family_arm_a8_Cache_branchPredictionEnabled__C)
                  8000fcdc    00000018     app_pea8fnv.oea8fnv (.const:ti_sysbios_gates_GateHwi_Object__PARAMS__C)
                  8000fcf4    00000018     app_pea8fnv.oea8fnv (.const:ti_sysbios_gates_GateMutex_Object__PARAMS__C)
                  8000fd0c    00000018     app_pea8fnv.oea8fnv (.const:ti_sysbios_knl_Queue_Object__PARAMS__C)
                  8000fd24    00000011     ti.targets.arm.rtsarm.aea8fnv : System.oea8fnv (.const:.string)
                  8000fd35    00000001     app_pea8fnv.oea8fnv (.const:xdc_runtime_Error_policy__C)
                  8000fd36    00000010     app_pea8fnv.oea8fnv (.const:ti_sysbios_family_arm_a8_Mmu_defaultAttrs__C)
                  8000fd46    00000002     app_pea8fnv.oea8fnv (.const:ti_sysbios_family_arm_a8_Cache_enableCache__C)
                  8000fd48    0000000c     app_pea8fnv.oea8fnv (.const:xdc_runtime_Startup_firstFxns__A)
                  8000fd54    00000008     app_pea8fnv.oea8fnv (.const:ti_sysbios_knl_Idle_funcList__C)
                  8000fd5c    00000008     app_pea8fnv.oea8fnv (.const:xdc_runtime_Startup_firstFxns__C)
                  8000fd64    00000008     app_pea8fnv.oea8fnv (.const:xdc_runtime_Startup_lastFxns__C)
                  8000fd6c    00000004     app_pea8fnv.oea8fnv (.const:ti_sysbios_family_arm_a8_Mmu_A_nullPointer__C)
                  8000fd70    00000004     app_pea8fnv.oea8fnv (.const:ti_sysbios_family_arm_a8_Mmu_A_unknownDescType__C)
                  8000fd74    00000004     app_pea8fnv.oea8fnv (.const:ti_sysbios_family_arm_a8_Mmu_Module__diagsEnabled__C)
                  8000fd78    00000004     app_pea8fnv.oea8fnv (.const:ti_sysbios_family_arm_a8_Mmu_Module__diagsIncluded__C)
                  8000fd7c    00000004     app_pea8fnv.oea8fnv (.const:ti_sysbios_family_arm_a8_Mmu_Module__diagsMask__C)
                  8000fd80    00000004     app_pea8fnv.oea8fnv (.const:ti_sysbios_family_arm_a8_intcps_Hwi_E_undefined__C)
                  8000fd84    00000004     app_pea8fnv.oea8fnv (.const:ti_sysbios_family_arm_a8_intcps_Hwi_LD_end__C)
                  8000fd88    00000004     app_pea8fnv.oea8fnv (.const:ti_sysbios_family_arm_a8_intcps_Hwi_LM_begin__C)
                  8000fd8c    00000004     app_pea8fnv.oea8fnv (.const:ti_sysbios_family_arm_a8_intcps_Hwi_Module__diagsEnabled__C)
                  8000fd90    00000004     app_pea8fnv.oea8fnv (.const:ti_sysbios_family_arm_a8_intcps_Hwi_Module__diagsIncluded__C)
                  8000fd94    00000004     app_pea8fnv.oea8fnv (.const:ti_sysbios_family_arm_a8_intcps_Hwi_Module__diagsMask__C)
                  8000fd98    00000004     app_pea8fnv.oea8fnv (.const:ti_sysbios_family_arm_a8_intcps_Hwi_Module__loggerFxn1__C)
                  8000fd9c    00000004     app_pea8fnv.oea8fnv (.const:ti_sysbios_family_arm_a8_intcps_Hwi_Module__loggerFxn8__C)
                  8000fda0    00000004     app_pea8fnv.oea8fnv (.const:ti_sysbios_family_arm_a8_intcps_Hwi_Module__loggerObj__C)
                  8000fda4    00000004     app_pea8fnv.oea8fnv (.const:ti_sysbios_family_arm_a8_intcps_Hwi_NUM_PRIORITIES__C)
                  8000fda8    00000004     app_pea8fnv.oea8fnv (.const:ti_sysbios_family_arm_a8_intcps_Hwi_taskDisable__C)
                  8000fdac    00000004     app_pea8fnv.oea8fnv (.const:ti_sysbios_family_arm_a8_intcps_Hwi_taskRestoreHwi__C)
                  8000fdb0    00000004     app_pea8fnv.oea8fnv (.const:ti_sysbios_family_arm_exc_Exception_E_dataAbort__C)
                  8000fdb4    00000004     app_pea8fnv.oea8fnv (.const:ti_sysbios_family_arm_exc_Exception_E_prefetchAbort__C)
                  8000fdb8    00000004     app_pea8fnv.oea8fnv (.const:ti_sysbios_family_arm_exc_Exception_E_swi__C)
                  8000fdbc    00000004     app_pea8fnv.oea8fnv (.const:ti_sysbios_family_arm_exc_Exception_E_undefinedInstruction__C)
                  8000fdc0    00000004     app_pea8fnv.oea8fnv (.const:ti_sysbios_family_arm_exc_Exception_excHookFuncs__A)
                  8000fdc4    00000004     app_pea8fnv.oea8fnv (.const:ti_sysbios_family_arm_exc_Exception_excHookFuncs__C)
                  8000fdc8    00000004     app_pea8fnv.oea8fnv (.const:ti_sysbios_gates_GateMutex_A_badContext__C)
                  8000fdcc    00000004     app_pea8fnv.oea8fnv (.const:ti_sysbios_gates_GateMutex_Instance_State_sem__O)
                  8000fdd0    00000004     app_pea8fnv.oea8fnv (.const:ti_sysbios_gates_GateMutex_Module__diagsEnabled__C)
                  8000fdd4    00000004     app_pea8fnv.oea8fnv (.const:ti_sysbios_gates_GateMutex_Module__diagsIncluded__C)
                  8000fdd8    00000004     app_pea8fnv.oea8fnv (.const:ti_sysbios_gates_GateMutex_Module__diagsMask__C)
                  8000fddc    00000004     app_pea8fnv.oea8fnv (.const:ti_sysbios_hal_Hwi_E_stackOverflow__C)
                  8000fde0    00000004     app_pea8fnv.oea8fnv (.const:ti_sysbios_heaps_HeapMem_A_align__C)
                  8000fde4    00000004     app_pea8fnv.oea8fnv (.const:ti_sysbios_heaps_HeapMem_A_heapSize__C)
                  8000fde8    00000004     app_pea8fnv.oea8fnv (.const:ti_sysbios_heaps_HeapMem_A_invalidFree__C)
                  8000fdec    00000004     app_pea8fnv.oea8fnv (.const:ti_sysbios_heaps_HeapMem_A_zeroBlock__C)
                  8000fdf0    00000004     app_pea8fnv.oea8fnv (.const:ti_sysbios_heaps_HeapMem_E_memory__C)
                  8000fdf4    00000004     app_pea8fnv.oea8fnv (.const:ti_sysbios_heaps_HeapMem_Module__diagsEnabled__C)
                  8000fdf8    00000004     app_pea8fnv.oea8fnv (.const:ti_sysbios_heaps_HeapMem_Module__diagsIncluded__C)
                  8000fdfc    00000004     app_pea8fnv.oea8fnv (.const:ti_sysbios_heaps_HeapMem_Module__diagsMask__C)
                  8000fe00    00000004     app_pea8fnv.oea8fnv (.const:ti_sysbios_heaps_HeapMem_Module__gateObj__C)
                  8000fe04    00000004     app_pea8fnv.oea8fnv (.const:ti_sysbios_heaps_HeapMem_Object__count__C)
                  8000fe08    00000004     app_pea8fnv.oea8fnv (.const:ti_sysbios_heaps_HeapMem_reqAlign__C)
                  8000fe0c    00000004     app_pea8fnv.oea8fnv (.const:ti_sysbios_knl_Clock_LM_begin__C)
                  8000fe10    00000004     app_pea8fnv.oea8fnv (.const:ti_sysbios_knl_Clock_LM_tick__C)
                  8000fe14    00000004     app_pea8fnv.oea8fnv (.const:ti_sysbios_knl_Clock_LW_delayed__C)
                  8000fe18    00000004     app_pea8fnv.oea8fnv (.const:ti_sysbios_knl_Clock_Module_State_clockQ__O)
                  8000fe1c    00000004     app_pea8fnv.oea8fnv (.const:ti_sysbios_knl_Clock_Module__diagsEnabled__C)
                  8000fe20    00000004     app_pea8fnv.oea8fnv (.const:ti_sysbios_knl_Clock_Module__diagsIncluded__C)
                  8000fe24    00000004     app_pea8fnv.oea8fnv (.const:ti_sysbios_knl_Clock_Module__diagsMask__C)
                  8000fe28    00000004     app_pea8fnv.oea8fnv (.const:ti_sysbios_knl_Clock_Module__loggerFxn1__C)
                  8000fe2c    00000004     app_pea8fnv.oea8fnv (.const:ti_sysbios_knl_Clock_Module__loggerFxn2__C)
                  8000fe30    00000004     app_pea8fnv.oea8fnv (.const:ti_sysbios_knl_Clock_Module__loggerObj__C)
                  8000fe34    00000004     app_pea8fnv.oea8fnv (.const:ti_sysbios_knl_Idle_funcList__A)
                  8000fe38    00000004     app_pea8fnv.oea8fnv (.const:ti_sysbios_knl_Semaphore_A_badContext__C)
                  8000fe3c    00000004     app_pea8fnv.oea8fnv (.const:ti_sysbios_knl_Semaphore_A_noEvents__C)
                  8000fe40    00000004     app_pea8fnv.oea8fnv (.const:ti_sysbios_knl_Semaphore_A_overflow__C)
                  8000fe44    00000004     app_pea8fnv.oea8fnv (.const:ti_sysbios_knl_Semaphore_A_pendTaskDisabled__C)
                  8000fe48    00000004     app_pea8fnv.oea8fnv (.const:ti_sysbios_knl_Semaphore_Instance_State_pendQ__O)
                  8000fe4c    00000004     app_pea8fnv.oea8fnv (.const:ti_sysbios_knl_Semaphore_LM_pend__C)
                  8000fe50    00000004     app_pea8fnv.oea8fnv (.const:ti_sysbios_knl_Semaphore_LM_post__C)
                  8000fe54    00000004     app_pea8fnv.oea8fnv (.const:ti_sysbios_knl_Semaphore_Module__diagsEnabled__C)
                  8000fe58    00000004     app_pea8fnv.oea8fnv (.const:ti_sysbios_knl_Semaphore_Module__diagsIncluded__C)
                  8000fe5c    00000004     app_pea8fnv.oea8fnv (.const:ti_sysbios_knl_Semaphore_Module__diagsMask__C)
                  8000fe60    00000004     app_pea8fnv.oea8fnv (.const:ti_sysbios_knl_Semaphore_Module__loggerFxn2__C)
                  8000fe64    00000004     app_pea8fnv.oea8fnv (.const:ti_sysbios_knl_Semaphore_Module__loggerFxn4__C)
                  8000fe68    00000004     app_pea8fnv.oea8fnv (.const:ti_sysbios_knl_Semaphore_Module__loggerObj__C)
                  8000fe6c    00000004     app_pea8fnv.oea8fnv (.const:ti_sysbios_knl_Swi_LD_end__C)
                  8000fe70    00000004     app_pea8fnv.oea8fnv (.const:ti_sysbios_knl_Swi_LM_begin__C)
                  8000fe74    00000004     app_pea8fnv.oea8fnv (.const:ti_sysbios_knl_Swi_LM_post__C)
                  8000fe78    00000004     app_pea8fnv.oea8fnv (.const:ti_sysbios_knl_Swi_Module__diagsEnabled__C)
                  8000fe7c    00000004     app_pea8fnv.oea8fnv (.const:ti_sysbios_knl_Swi_Module__diagsIncluded__C)
                  8000fe80    00000004     app_pea8fnv.oea8fnv (.const:ti_sysbios_knl_Swi_Module__diagsMask__C)
                  8000fe84    00000004     app_pea8fnv.oea8fnv (.const:ti_sysbios_knl_Swi_Module__loggerFxn1__C)
                  8000fe88    00000004     app_pea8fnv.oea8fnv (.const:ti_sysbios_knl_Swi_Module__loggerFxn4__C)
                  8000fe8c    00000004     app_pea8fnv.oea8fnv (.const:ti_sysbios_knl_Swi_Module__loggerObj__C)
                  8000fe90    00000004     app_pea8fnv.oea8fnv (.const:ti_sysbios_knl_Swi_Object__count__C)
                  8000fe94    00000004     app_pea8fnv.oea8fnv (.const:ti_sysbios_knl_Task_A_badPriority__C)
                  8000fe98    00000004     app_pea8fnv.oea8fnv (.const:ti_sysbios_knl_Task_A_badTaskState__C)
                  8000fe9c    00000004     app_pea8fnv.oea8fnv (.const:ti_sysbios_knl_Task_A_badThreadType__C)
                  8000fea0    00000004     app_pea8fnv.oea8fnv (.const:ti_sysbios_knl_Task_A_badTimeout__C)
                  8000fea4    00000004     app_pea8fnv.oea8fnv (.const:ti_sysbios_knl_Task_A_noPendElem__C)
                  8000fea8    00000004     app_pea8fnv.oea8fnv (.const:ti_sysbios_knl_Task_A_sleepTaskDisabled__C)
                  8000feac    00000004     app_pea8fnv.oea8fnv (.const:ti_sysbios_knl_Task_E_spOutOfBounds__C)
                  8000feb0    00000004     app_pea8fnv.oea8fnv (.const:ti_sysbios_knl_Task_E_stackOverflow__C)
                  8000feb4    00000004     app_pea8fnv.oea8fnv (.const:ti_sysbios_knl_Task_LD_block__C)
                  8000feb8    00000004     app_pea8fnv.oea8fnv (.const:ti_sysbios_knl_Task_LD_exit__C)
                  8000febc    00000004     app_pea8fnv.oea8fnv (.const:ti_sysbios_knl_Task_LD_ready__C)
                  8000fec0    00000004     app_pea8fnv.oea8fnv (.const:ti_sysbios_knl_Task_LM_sleep__C)
                  8000fec4    00000004     app_pea8fnv.oea8fnv (.const:ti_sysbios_knl_Task_LM_switch__C)
                  8000fec8    00000004     app_pea8fnv.oea8fnv (.const:ti_sysbios_knl_Task_Module_State_inactiveQ__O)
                  8000fecc    00000004     app_pea8fnv.oea8fnv (.const:ti_sysbios_knl_Task_Module__diagsEnabled__C)
                  8000fed0    00000004     app_pea8fnv.oea8fnv (.const:ti_sysbios_knl_Task_Module__diagsIncluded__C)
                  8000fed4    00000004     app_pea8fnv.oea8fnv (.const:ti_sysbios_knl_Task_Module__diagsMask__C)
                  8000fed8    00000004     app_pea8fnv.oea8fnv (.const:ti_sysbios_knl_Task_Module__loggerFxn2__C)
                  8000fedc    00000004     app_pea8fnv.oea8fnv (.const:ti_sysbios_knl_Task_Module__loggerFxn4__C)
                  8000fee0    00000004     app_pea8fnv.oea8fnv (.const:ti_sysbios_knl_Task_Module__loggerObj__C)
                  8000fee4    00000004     app_pea8fnv.oea8fnv (.const:ti_sysbios_knl_Task_Object__count__C)
                  8000fee8    00000004     app_pea8fnv.oea8fnv (.const:ti_sysbios_knl_Task_allBlockedFunc__C)
                  8000feec    00000004     app_pea8fnv.oea8fnv (.const:ti_sysbios_knl_Task_defaultStackHeap__C)
                  8000fef0    00000004     app_pea8fnv.oea8fnv (.const:ti_sysbios_knl_Task_defaultStackSize__C)
                  8000fef4    00000004     app_pea8fnv.oea8fnv (.const:ti_sysbios_knl_Task_numConstructedTasks__C)
                  8000fef8    00000004     app_pea8fnv.oea8fnv (.const:ti_sysbios_timers_dmtimer_Timer_E_cannotSupport__C)
                  8000fefc    00000004     app_pea8fnv.oea8fnv (.const:ti_sysbios_timers_dmtimer_Timer_E_freqMismatch__C)
                  8000ff00    00000004     app_pea8fnv.oea8fnv (.const:ti_sysbios_timers_dmtimer_Timer_Module__diagsEnabled__C)
                  8000ff04    00000004     app_pea8fnv.oea8fnv (.const:ti_sysbios_timers_dmtimer_Timer_Module__diagsIncluded__C)
                  8000ff08    00000004     app_pea8fnv.oea8fnv (.const:ti_sysbios_timers_dmtimer_Timer_Module__diagsMask__C)
                  8000ff0c    00000004     app_pea8fnv.oea8fnv (.const:ti_sysbios_timers_dmtimer_Timer_numTimerDevices__C)
                  8000ff10    00000004     app_pea8fnv.oea8fnv (.const:xdc_runtime_Assert_E_assertFailed__C)
                  8000ff14    00000004     app_pea8fnv.oea8fnv (.const:xdc_runtime_Core_A_initializedParams__C)
                  8000ff18    00000004     app_pea8fnv.oea8fnv (.const:xdc_runtime_Core_Module__diagsEnabled__C)
                  8000ff1c    00000004     app_pea8fnv.oea8fnv (.const:xdc_runtime_Core_Module__diagsIncluded__C)
                  8000ff20    00000004     app_pea8fnv.oea8fnv (.const:xdc_runtime_Core_Module__diagsMask__C)
                  8000ff24    00000004     app_pea8fnv.oea8fnv (.const:xdc_runtime_Error_E_memory__C)
                  8000ff28    00000004     app_pea8fnv.oea8fnv (.const:xdc_runtime_Error_Module__diagsEnabled__C)
                  8000ff2c    00000004     app_pea8fnv.oea8fnv (.const:xdc_runtime_Error_Module__diagsIncluded__C)
                  8000ff30    00000004     app_pea8fnv.oea8fnv (.const:xdc_runtime_Error_Module__diagsMask__C)
                  8000ff34    00000004     app_pea8fnv.oea8fnv (.const:xdc_runtime_Error_Module__loggerFxn8__C)
                  8000ff38    00000004     app_pea8fnv.oea8fnv (.const:xdc_runtime_Error_Module__loggerObj__C)
                  8000ff3c    00000004     app_pea8fnv.oea8fnv (.const:xdc_runtime_Error_policyFxn__C)
                  8000ff40    00000004     app_pea8fnv.oea8fnv (.const:xdc_runtime_Error_raiseHook__C)
                  8000ff44    00000004     app_pea8fnv.oea8fnv (.const:xdc_runtime_IFilterLogger_Interface__BASE__C)
                  8000ff48    00000004     app_pea8fnv.oea8fnv (.const:xdc_runtime_IGateProvider_Interface__BASE__C)
                  8000ff4c    00000004     app_pea8fnv.oea8fnv (.const:xdc_runtime_IHeap_Interface__BASE__C)
                  8000ff50    00000004     app_pea8fnv.oea8fnv (.const:xdc_runtime_ILogger_Interface__BASE__C)
                  8000ff54    00000004     app_pea8fnv.oea8fnv (.const:xdc_runtime_IModule_Interface__BASE__C)
                  8000ff58    00000004     app_pea8fnv.oea8fnv (.const:xdc_runtime_Log_L_error__C)
                  8000ff5c    00000004     app_pea8fnv.oea8fnv (.const:xdc_runtime_LoggerBuf_E_badLevel__C)
                  8000ff60    00000004     app_pea8fnv.oea8fnv (.const:xdc_runtime_LoggerBuf_Module__gateObj__C)
                  8000ff64    00000004     app_pea8fnv.oea8fnv (.const:xdc_runtime_LoggerBuf_Object__count__C)
                  8000ff68    00000004     app_pea8fnv.oea8fnv (.const:xdc_runtime_LoggerBuf_statusLogger__C)
                  8000ff6c    00000004     app_pea8fnv.oea8fnv (.const:xdc_runtime_Memory_defaultHeapInstance__C)
                  8000ff70    00000004     app_pea8fnv.oea8fnv (.const:xdc_runtime_Startup_execImpl__C)
                  8000ff74    00000004     app_pea8fnv.oea8fnv (.const:xdc_runtime_Startup_maxPasses__C)
                  8000ff78    00000004     app_pea8fnv.oea8fnv (.const:xdc_runtime_Startup_sfxnRts__C)
                  8000ff7c    00000004     app_pea8fnv.oea8fnv (.const:xdc_runtime_Startup_sfxnTab__C)
                  8000ff80    00000004     app_pea8fnv.oea8fnv (.const:xdc_runtime_SysMin_bufSize__C)
                  8000ff84    00000004     app_pea8fnv.oea8fnv (.const:xdc_runtime_SysMin_outputFunc__C)
                  8000ff88    00000004     app_pea8fnv.oea8fnv (.const:xdc_runtime_System_Module__gateObj__C)
                  8000ff8c    00000004     app_pea8fnv.oea8fnv (.const:xdc_runtime_System_abortFxn__C)
                  8000ff90    00000004     app_pea8fnv.oea8fnv (.const:xdc_runtime_System_exitFxn__C)
                  8000ff94    00000004     app_pea8fnv.oea8fnv (.const:xdc_runtime_System_extendFxn__C)
                  8000ff98    00000004     app_pea8fnv.oea8fnv (.const:xdc_runtime_System_maxAtexitHandlers__C)
                  8000ff9c    00000004     app_pea8fnv.oea8fnv (.const:xdc_runtime_Text_charTab__C)
                  8000ffa0    00000004     app_pea8fnv.oea8fnv (.const:xdc_runtime_Text_nameEmpty__C)
                  8000ffa4    00000004     app_pea8fnv.oea8fnv (.const:xdc_runtime_Text_nameStatic__C)
                  8000ffa8    00000004     app_pea8fnv.oea8fnv (.const:xdc_runtime_Text_nameUnknown__C)
                  8000ffac    00000004     app_pea8fnv.oea8fnv (.const:xdc_runtime_Text_nodeTab__C)
                  8000ffb0    00000004     app_pea8fnv.oea8fnv (.const:xdc_runtime_Text_visitRopeFxn__C)
                  8000ffb4    00000002     app_pea8fnv.oea8fnv (.const:ti_sysbios_family_arm_a8_Cache_unlockL2Cache__C)
                  8000ffb6    00000002     app_pea8fnv.oea8fnv (.const:ti_sysbios_family_arm_a8_Mmu_Module__id__C)
                  8000ffb8    00000002     app_pea8fnv.oea8fnv (.const:ti_sysbios_family_arm_a8_Mmu_enableMMU__C)
                  8000ffba    00000002     app_pea8fnv.oea8fnv (.const:ti_sysbios_family_arm_a8_intcps_Hwi_Module__id__C)
                  8000ffbc    00000002     app_pea8fnv.oea8fnv (.const:ti_sysbios_family_arm_a8_intcps_Hwi_Module__loggerDefined__C)
                  8000ffbe    00000002     app_pea8fnv.oea8fnv (.const:ti_sysbios_family_arm_exc_Exception_Module__id__C)
                  8000ffc0    00000002     app_pea8fnv.oea8fnv (.const:ti_sysbios_gates_GateMutex_Module__id__C)
                  8000ffc2    00000002     app_pea8fnv.oea8fnv (.const:ti_sysbios_hal_Hwi_Module__id__C)
                  8000ffc4    00000002     app_pea8fnv.oea8fnv (.const:ti_sysbios_heaps_HeapMem_Module__id__C)
                  8000ffc6    00000002     app_pea8fnv.oea8fnv (.const:ti_sysbios_knl_Clock_Module__id__C)
                  8000ffc8    00000002     app_pea8fnv.oea8fnv (.const:ti_sysbios_knl_Clock_Module__loggerDefined__C)
                  8000ffca    00000002     app_pea8fnv.oea8fnv (.const:ti_sysbios_knl_Semaphore_Module__id__C)
                  8000ffcc    00000002     app_pea8fnv.oea8fnv (.const:ti_sysbios_knl_Semaphore_Module__loggerDefined__C)
                  8000ffce    00000002     app_pea8fnv.oea8fnv (.const:ti_sysbios_knl_Swi_Module__id__C)
                  8000ffd0    00000002     app_pea8fnv.oea8fnv (.const:ti_sysbios_knl_Swi_Module__loggerDefined__C)
                  8000ffd2    00000002     app_pea8fnv.oea8fnv (.const:ti_sysbios_knl_Task_Module__id__C)
                  8000ffd4    00000002     app_pea8fnv.oea8fnv (.const:ti_sysbios_knl_Task_Module__loggerDefined__C)
                  8000ffd6    00000002     app_pea8fnv.oea8fnv (.const:ti_sysbios_knl_Task_initStackFlag__C)
                  8000ffd8    00000002     app_pea8fnv.oea8fnv (.const:ti_sysbios_timers_dmtimer_Timer_Module__id__C)
                  8000ffda    00000002     app_pea8fnv.oea8fnv (.const:ti_sysbios_timers_dmtimer_Timer_checkFrequency__C)
                  8000ffdc    00000002     app_pea8fnv.oea8fnv (.const:ti_sysbios_timers_dmtimer_Timer_startupNeeded__C)
                  8000ffde    00000002     app_pea8fnv.oea8fnv (.const:xdc_runtime_Core_Module__id__C)
                  8000ffe0    00000002     app_pea8fnv.oea8fnv (.const:xdc_runtime_Error_Module__loggerDefined__C)
                  8000ffe2    00000002     app_pea8fnv.oea8fnv (.const:xdc_runtime_Error_maxDepth__C)
                  8000ffe4    00000002     app_pea8fnv.oea8fnv (.const:xdc_runtime_LoggerBuf_Module__id__C)
                  8000ffe6    00000002     app_pea8fnv.oea8fnv (.const:xdc_runtime_LoggerBuf_filterByLevel__C)
                  8000ffe8    00000002     app_pea8fnv.oea8fnv (.const:xdc_runtime_Memory_Module__id__C)
                  8000ffea    00000002     app_pea8fnv.oea8fnv (.const:xdc_runtime_SysMin_flushAtExit__C)
                  8000ffec    00000002     app_pea8fnv.oea8fnv (.const:xdc_runtime_Text_charCnt__C)
                  8000ffee    00000002     app_pea8fnv.oea8fnv (.const:xdc_runtime_Text_isLoaded__C)
                  8000fff0    00000002     app_pea8fnv.oea8fnv (.const:xdc_runtime_Text_registryModsLastId__C)
                  8000fff2    00000002     app_pea8fnv.oea8fnv (.const:xdc_runtime_Text_unnamedModsLastId__C)

.data.1    0    8000fff4    0000000c     UNINITIALIZED
                  8000fff4    00000008     rtsv7A8_A_le_n_v3_eabi.lib : _lock.obj (.data)
                  8000fffc    00000004                                : stkdepth_vars.obj (.data)

.const.3   0    80014000    0000194e     
                  80014000    0000194e     app_pea8fnv.oea8fnv (.const:xdc_runtime_Text_charTab__A)

.data.2    0    80017950    0000093c     UNINITIALIZED
                  80017950    00000250     app_pea8fnv.oea8fnv (.data:ti_sysbios_family_arm_a8_intcps_Hwi_Module__state__V)
                  80017ba0    00000198     app_pea8fnv.oea8fnv (.data)
                  80017d38    00000180     gpmc_fpga.obj (.data:GpmcMux)
                  80017eb8    00000080     app_pea8fnv.oea8fnv (.data:ti_sysbios_knl_Swi_Module_State_0_readyQ__A)
                  80017f38    00000080     app_pea8fnv.oea8fnv (.data:ti_sysbios_knl_Task_Module_State_0_readyQ__A)
                  80017fb8    0000005c     app_pea8fnv.oea8fnv (.data:ti_sysbios_timers_dmtimer_Timer_Object__table__V)
                  80018014    00000058     main.obj (.data:applMmuEntries)
                  8001806c    0000004c     app_pea8fnv.oea8fnv (.data:ti_sysbios_knl_Task_Object__table__V)
                  800180b8    00000048     app_pea8fnv.oea8fnv (.data:ti_sysbios_timers_dmtimer_Timer_Module_State_0_device__A)
                  80018100    00000044     app_pea8fnv.oea8fnv (.data:ti_sysbios_knl_Task_Module__state__V)
                  80018144    00000038     app_pea8fnv.oea8fnv (.data:ti_sysbios_gates_GateMutex_Object__table__V)
                  8001817c    00000034     app_pea8fnv.oea8fnv (.data:ti_sysbios_family_arm_a8_Cache_Module__state__V)
                  800181b0    00000030     app_pea8fnv.oea8fnv (.data:ti_sysbios_knl_Swi_Object__table__V)
                  800181e0    00000030     app_pea8fnv.oea8fnv (.data:ti_sysbios_timers_dmtimer_Timer_Module_State_0_intFreqs__A)
                  80018210    0000002c     app_pea8fnv.oea8fnv (.data:ti_sysbios_knl_Clock_Module__state__V)
                  8001823c    00000024     app_pea8fnv.oea8fnv (.data:ti_sysbios_BIOS_Module__state__V)
                  80018260    00000024     app_pea8fnv.oea8fnv (.data:xdc_runtime_LoggerBuf_Object__table__V)
                  80018284    00000008     rtsv7A8_A_le_n_v3_eabi.lib : exit.obj (.data)

.vecs      0    80018400    00000040     
                  80018400    00000040     app_pea8fnv.oea8fnv (.vecs)

xdc.meta   0    80000000    000000e4     COPY SECTION
                  80000000    000000e4     app_pea8fnv.oea8fnv (xdc.meta)


LINKER GENERATED COPY TABLES

__TI_cinit_table @ 80018b50 records: 3, size/record: 8, table size: 24
	.data.2: load addr=80018440, load size=000006e5 bytes, run addr=80017950, run size=0000093c bytes, compression=rle
	.data.1: load addr=80018b28, load size=00000011 bytes, run addr=8000fff4, run size=0000000c bytes, compression=rle
	.bss: load addr=80018b48, load size=00000008 bytes, run addr=8000b808, run size=00004128 bytes, compression=zero_init


LINKER GENERATED HANDLER TABLE

__TI_handler_table @ 80018b3c records: 3, size/record: 4, table size: 12
	index: 0, handler: __TI_zero_init
	index: 1, handler: __TI_decompress_rle24
	index: 2, handler: __TI_decompress_none


GLOBAL SYMBOLS: SORTED ALPHABETICALLY BY Name 

address   name                                                                    
-------   ----                                                                    
80009910  C$$EXIT                                                                 
80008b58  C$$IO$$                                                                 
80000e4c  GPMCADVTimingConfig                                                     
80000ccc  GPMCAccessTypeSelect                                                    
80000820  GPMCAddrDataMuxProtocolSelect                                           
8000006c  GPMCAutoIdleConfig                                                      
80000ff8  GPMCBaseAddrSet                                                         
80000f8c  GPMCCSConfig                                                            
80000e18  GPMCCSTimingConfig                                                      
80000b1c  GPMCClkActivationTimeConfig                                             
80000b88  GPMCDevPageLenSet                                                       
800008f8  GPMCDevSizeSelect                                                       
8000088c  GPMCDevTypeSelect                                                       
800015c4  GPMCECCAlgoSelect                                                       
8000160c  GPMCECCBCHErrCorrectionCapSelect                                        
800016e4  GPMCECCBCHNumOfSectorsSelect                                            
80001b38  GPMCECCBCHResultGet                                                     
80001c68  GPMCECCBCHSWDataRead                                                    
80001c44  GPMCECCBCHSWDataWrite                                                   
80001654  GPMCECCBCHWrapModeValSet                                                
8000172c  GPMCECCCSSelect                                                         
8000169c  GPMCECCColumnSelect                                                     
80001798  GPMCECCDisable                                                          
80001774  GPMCECCEnable                                                           
80001b0c  GPMCECCResultGet                                                        
800017bc  GPMCECCResultRegClear                                                   
800017e0  GPMCECCResultRegSelect                                                  
800018c0  GPMCECCResultSizeSelect                                                 
80001824  GPMCECCSizeValSet                                                       
80000728  GPMCEmptyWriteBuffStatusGet                                             
80000408  GPMCErrAddrGet                                                          
80000478  GPMCErrStatusGet                                                        
80000450  GPMCErrSysCmdGet                                                        
8000042c  GPMCErrValStatusGet                                                     
8000074c  GPMCFclkDividerSelect                                                   
80000024  GPMCIdleModeSelect                                                      
800002c8  GPMCIntDisable                                                          
80000228  GPMCIntEnable                                                           
80000188  GPMCIntStatusClear                                                      
800000e4  GPMCIntStatusGet                                                        
80000614  GPMCLimitedAddrDevSupportConfig                                         
80001060  GPMCMaskAddrSet                                                         
800000c0  GPMCModuleResetStatusGet                                                
800000a4  GPMCModuleSoftReset                                                     
80001cac  GPMCMuxConfig1                                                          
80001dc4  GPMCMuxConfig2                                                          
80001e40  GPMCMuxConfig3                                                          
80001f04  GPMCMuxConfig4                                                          
80001fe0  GPMCMuxConfig5                                                          
8000205c  GPMCMuxConfig6                                                          
800020fc  GPMCMuxConfig7                                                          
80001100  GPMCNANDAddrWrite                                                       
80001168  GPMCNANDDataRead                                                        
80001134  GPMCNANDDataWrite                                                       
8000066c  GPMCNANDForcePostedWriteFeatureConfig                                   
80001390  GPMCPrefetchAccessCycleOptConfig                                        
8000119c  GPMCPrefetchAccessModeSelect                                            
80001348  GPMCPrefetchCSSelect                                                    
80001550  GPMCPrefetchCountValGet                                                 
800013d8  GPMCPrefetchCycleOptValSet                                              
800012dc  GPMCPrefetchEngineDisable                                               
800012b8  GPMCPrefetchEngineEnable                                                
800014f4  GPMCPrefetchEngineStart                                                 
8000152c  GPMCPrefetchEngineStatusGet                                             
80001510  GPMCPrefetchEngineStop                                                  
8000159c  GPMCPrefetchFifoPtrValGet                                               
80001574  GPMCPrefetchFifoThrldStatusGet                                          
80001300  GPMCPrefetchFifoThrldValSet                                             
80001420  GPMCPrefetchRRArbitrationConfig                                         
80001228  GPMCPrefetchSyncModeConfig                                              
800011e0  GPMCPrefetchSyncTypeSelect                                              
800014b0  GPMCPrefetchTrnsCntValSet                                               
80001270  GPMCPrefetchWaitPinSelect                                               
80001468  GPMCPrefetchWeightedPrioSet                                             
80000eb4  GPMCRdAccessAndCycleTimeTimingConfig                                    
80000c60  GPMCReadTypeSelect                                                      
80000000  GPMCRevisionGet                                                         
800010cc  GPMCSNANDCmdWrite                                                       
80000dac  GPMCSyncWrapBurstConfig                                                 
80001c8c  GPMCSystemConfig                                                        
800003b0  GPMCTimeOutFeatureConfig                                                
80000368  GPMCTimeOutStartValSet                                                  
800007b4  GPMCTimeParaGranularitySelect                                           
80000e80  GPMCWEAndOETimingConfig                                                 
800009d0  GPMCWaitMonitoringTimeSelect                                            
80000a3c  GPMCWaitPinMonitoringConfig                                             
80000500  GPMCWaitPinPolaritySelect                                               
80000964  GPMCWaitPinSelect                                                       
800006c4  GPMCWaitPinStatusGet                                                    
80000ee8  GPMCWrAccessAndWrDataOnADMUXBusTimingConfig                             
800005bc  GPMCWriteProtectPinLevelCtrl                                            
80000bf4  GPMCWriteTypeSelect                                                     
80000f4c  GPMCycle2CycleAndTurnArndTimeTimingConfig                               
8000213c  GpmcInitial                                                             
80017d38  GpmcMux                                                                 
80002268  GpmcReadFpga                                                            
80002200  GpmcWriteFpga                                                           
80002dfc  HOSTclock                                                               
80002d94  HOSTclose                                                               
80002d2c  HOSTgetenv                                                              
80002c8c  HOSTlseek                                                               
80002c00  HOSTopen                                                                
80002b7c  HOSTread                                                                
80002ae4  HOSTrename                                                              
80002a84  HOSTtime                                                                
80002a20  HOSTunlink                                                              
8000299c  HOSTwrite                                                               
8000b7bc  LoggerBuf_instanceStartup                                               
8000936d  MMUInit                                                                 
8000a83d  PRUSSPinMuxConfig                                                       
8000a80d  PinMuxConfig                                                            
UNDEFED   SHT$$INIT_ARRAY$$Base                                                   
UNDEFED   SHT$$INIT_ARRAY$$Limit                                                  
8001806c  TSK_idle                                                                
80000000  __ASM__                                                                 
8000f808  __CIOBUF_                                                               
8000005c  __ISA__                                                                 
8000006e  __PLAT__                                                                
80017950  __STACK_END                                                             
00002000  __STACK_SIZE                                                            
80000094  __TARG__                                                                
80018b50  __TI_CINIT_Base                                                         
80018b68  __TI_CINIT_Limit                                                        
80018b3c  __TI_Handler_Table_Base                                                 
80018b48  __TI_Handler_Table_Limit                                                
8000823c  __TI_auto_init                                                          
80018284  __TI_cleanup_ptr                                                        
8000b508  __TI_decompress_none                                                    
8000b754  __TI_decompress_rle24                                                   
80018288  __TI_dtors_ptr                                                          
80008b60  __TI_readmsg                                                            
80018440  __TI_static_base__                                                      
80008b10  __TI_writemsg                                                           
8000b634  __TI_zero_init                                                          
800000bc  __TRDR__                                                                
800089b0  __aeabi_memclr                                                          
800089b0  __aeabi_memclr4                                                         
800089b0  __aeabi_memclr8                                                         
800069fc  __aeabi_memcpy                                                          
800069fc  __aeabi_memcpy4                                                         
800069fc  __aeabi_memcpy8                                                         
800089b4  __aeabi_memset                                                          
800089b4  __aeabi_memset4                                                         
800089b4  __aeabi_memset8                                                         
80007e74  __aeabi_uidiv                                                           
80007e74  __aeabi_uidivmod                                                        
800049dc  __aeabi_uldivmod                                                        
ffffffff  __binit__                                                               
ffffffff  __c_args__                                                              
80015950  __stack                                                                 
8000b744  __xdc__init                                                             
80017d34  __xdc__init__addr                                                       
8000b17c  _args_main                                                              
00000000  _argsize                                                                
80009988  _c_int00                                                                
8000fff4  _lock                                                                   
8000b0e4  _nop                                                                    
8000b0d8  _register_lock                                                          
8000b0cc  _register_unlock                                                        
8000fff8  _unlock                                                                 
80009918  abort                                                                   
80018014  applMmuEntries                                                          
ffffffff  binit                                                                   
8000950c  copy_in                                                                 
80009924  exit                                                                    
80005450  main                                                                    
8000fffc  main_func_sp                                                            
800069fc  memcpy                                                                  
800089c0  memset                                                                  
8000b3d8  strcpy                                                                  
8000b238  strlen                                                                  
80005400  taskFxn                                                                 
8001823c  ti_sysbios_BIOS_Module__state__V                                        
8000ae5c  ti_sysbios_BIOS_RtsGateProxy_Handle__label__S                           
8000ab44  ti_sysbios_BIOS_RtsGateProxy_Object__delete__S                          
8000b7c0  ti_sysbios_BIOS_RtsGateProxy_enter__E                                   
8000b7c4  ti_sysbios_BIOS_RtsGateProxy_leave__E                                   
8000b79c  ti_sysbios_BIOS_RtsGateProxy_query__E                                   
8000a6b8  ti_sysbios_BIOS_atExitFunc__I                                           
8000aaa8  ti_sysbios_BIOS_errorRaiseHook__I                                       
8000b19c  ti_sysbios_BIOS_exitFunc__I                                             
8000b3f0  ti_sysbios_BIOS_exit__E                                                 
8000b644  ti_sysbios_BIOS_getCpuFreq__E                                           
8000b7c8  ti_sysbios_BIOS_nullFunc__I                                             
8000aadc  ti_sysbios_BIOS_registerRTSLock__I                                      
8000ab10  ti_sysbios_BIOS_removeRTSLock__I                                        
8000ace0  ti_sysbios_BIOS_rtsLock__I                                              
8000af64  ti_sysbios_BIOS_rtsUnlock__I                                            
8000b408  ti_sysbios_BIOS_setThreadType__E                                        
8000af8c  ti_sysbios_BIOS_startFunc__I                                            
8000b420  ti_sysbios_BIOS_start__E                                                
8000b75c  ti_sysbios_family_arm_TaskSupport_Module__startupDone__S                
80009818  ti_sysbios_family_arm_TaskSupport_buildTaskStack                        
8000b51c  ti_sysbios_family_arm_TaskSupport_checkStack__E                         
8000b654  ti_sysbios_family_arm_TaskSupport_getStackAlignment__E                  
8000b21c  ti_sysbios_family_arm_TaskSupport_glue                                  
8000b804  ti_sysbios_family_arm_TaskSupport_stackAlignment__C                     
80009ca4  ti_sysbios_family_arm_TaskSupport_start__E                              
8000b3c0  ti_sysbios_family_arm_TaskSupport_swap__E                               
8001817c  ti_sysbios_family_arm_a8_Cache_Module__state__V                         
8000fcda  ti_sysbios_family_arm_a8_Cache_branchPredictionEnabled__C               
8000b254  ti_sysbios_family_arm_a8_Cache_disableBP__E                             
8000b270  ti_sysbios_family_arm_a8_Cache_disableL1d__I                            
8000b530  ti_sysbios_family_arm_a8_Cache_disableL1p__I                            
8000b664  ti_sysbios_family_arm_a8_Cache_disableL2__I                             
80009e44  ti_sysbios_family_arm_a8_Cache_disable__E                               
8000b28c  ti_sysbios_family_arm_a8_Cache_enableBP__E                              
8000fd46  ti_sysbios_family_arm_a8_Cache_enableCache__C                           
8000b674  ti_sysbios_family_arm_a8_Cache_enableL1d__I                             
8000b544  ti_sysbios_family_arm_a8_Cache_enableL1p__I                             
8000b684  ti_sysbios_family_arm_a8_Cache_enableL2__I                              
8000a84c  ti_sysbios_family_arm_a8_Cache_enable__E                                
8000b714  ti_sysbios_family_arm_a8_Cache_getCacheLevelInfo__I                     
8000aa38  ti_sysbios_family_arm_a8_Cache_getEnabled__E                            
8000b764  ti_sysbios_family_arm_a8_Cache_getLockdownReg__I                        
80009124  ti_sysbios_family_arm_a8_Cache_invL1dAll__E                             
8000b76c  ti_sysbios_family_arm_a8_Cache_invL1pAll__E                             
8000b774  ti_sysbios_family_arm_a8_Cache_setLockdownReg__I                        
80006b7c  ti_sysbios_family_arm_a8_Cache_startup__I                               
8000ffb4  ti_sysbios_family_arm_a8_Cache_unlockL2Cache__C                         
800091b8  ti_sysbios_family_arm_a8_Cache_wbInvAll__E                              
8000fd6c  ti_sysbios_family_arm_a8_Mmu_A_nullPointer__C                           
8000fd70  ti_sysbios_family_arm_a8_Mmu_A_unknownDescType__C                       
80010000  ti_sysbios_family_arm_a8_Mmu_Module_State_0_tableBuf__A                 
8000fd74  ti_sysbios_family_arm_a8_Mmu_Module__diagsEnabled__C                    
8000fd78  ti_sysbios_family_arm_a8_Mmu_Module__diagsIncluded__C                   
8000fd7c  ti_sysbios_family_arm_a8_Mmu_Module__diagsMask__C                       
8000ffb6  ti_sysbios_family_arm_a8_Mmu_Module__id__C                              
80017ba0  ti_sysbios_family_arm_a8_Mmu_Module__state__V                           
80009484  ti_sysbios_family_arm_a8_Mmu_Module_startup__E                          
8000fd36  ti_sysbios_family_arm_a8_Mmu_defaultAttrs__C                            
8000b15c  ti_sysbios_family_arm_a8_Mmu_disableAsm__I                              
8000a90c  ti_sysbios_family_arm_a8_Mmu_disable__E                                 
8000acb0  ti_sysbios_family_arm_a8_Mmu_enableAsm__I                               
8000ffb8  ti_sysbios_family_arm_a8_Mmu_enableMMU__C                               
80009b58  ti_sysbios_family_arm_a8_Mmu_enable__E                                  
80007704  ti_sysbios_family_arm_a8_Mmu_initDescAttrs__E                           
80003db8  ti_sysbios_family_arm_a8_Mmu_initTableBuf__I                            
8000b4e0  ti_sysbios_family_arm_a8_Mmu_init__I                                    
8000b4f4  ti_sysbios_family_arm_a8_Mmu_isEnabled__E                               
8000b74c  ti_sysbios_family_arm_a8_Mmu_setDomainAccessCtrlReg__E                  
80004c94  ti_sysbios_family_arm_a8_Mmu_setFirstLevelDesc__E                       
80017ba4  ti_sysbios_family_arm_a8_TimestampProvider_Module__state__V             
8000b694  ti_sysbios_family_arm_a8_TimestampProvider_Module_startup__E            
8000a948  ti_sysbios_family_arm_a8_TimestampProvider_autoRefreshFxn__I            
8000b77c  ti_sysbios_family_arm_a8_TimestampProvider_get32__E                     
8000a590  ti_sysbios_family_arm_a8_TimestampProvider_get64__E                     
8000b644  ti_sysbios_family_arm_a8_TimestampProvider_getFreq__E                   
8000b2a8  ti_sysbios_family_arm_a8_TimestampProvider_initCCNT__I                  
8000fd80  ti_sysbios_family_arm_a8_intcps_Hwi_E_undefined__C                      
8000fd84  ti_sysbios_family_arm_a8_intcps_Hwi_LD_end__C                           
8000fd88  ti_sysbios_family_arm_a8_intcps_Hwi_LM_begin__C                         
8000f008  ti_sysbios_family_arm_a8_intcps_Hwi_Module_State_0_fiqStack__A          
8000fd8c  ti_sysbios_family_arm_a8_intcps_Hwi_Module__diagsEnabled__C             
8000fd90  ti_sysbios_family_arm_a8_intcps_Hwi_Module__diagsIncluded__C            
8000fd94  ti_sysbios_family_arm_a8_intcps_Hwi_Module__diagsMask__C                
8000ffba  ti_sysbios_family_arm_a8_intcps_Hwi_Module__id__C                       
8000ffbc  ti_sysbios_family_arm_a8_intcps_Hwi_Module__loggerDefined__C            
8000fd98  ti_sysbios_family_arm_a8_intcps_Hwi_Module__loggerFxn1__C               
8000fd9c  ti_sysbios_family_arm_a8_intcps_Hwi_Module__loggerFxn8__C               
8000fda0  ti_sysbios_family_arm_a8_intcps_Hwi_Module__loggerObj__C                
80017bac  ti_sysbios_family_arm_a8_intcps_Hwi_Module__root__V                     
8000afb4  ti_sysbios_family_arm_a8_intcps_Hwi_Module__startupDone__F              
8000afb4  ti_sysbios_family_arm_a8_intcps_Hwi_Module__startupDone__S              
80017950  ti_sysbios_family_arm_a8_intcps_Hwi_Module__state__V                    
80006cf4  ti_sysbios_family_arm_a8_intcps_Hwi_Module_startup__E                   
8000fda4  ti_sysbios_family_arm_a8_intcps_Hwi_NUM_PRIORITIES__C                   
80017bb4  ti_sysbios_family_arm_a8_intcps_Hwi_Object__table__V                    
8000b558  ti_sysbios_family_arm_a8_intcps_Hwi_clearInterrupt__E                   
8000805c  ti_sysbios_family_arm_a8_intcps_Hwi_disableInterrupt__E                 
800099fc  ti_sysbios_family_arm_a8_intcps_Hwi_dispatchFIQC__I                     
80005860  ti_sysbios_family_arm_a8_intcps_Hwi_dispatchIRQC__I                     
8000883c  ti_sysbios_family_arm_a8_intcps_Hwi_dispatchIRQ__I                      
8000814c  ti_sysbios_family_arm_a8_intcps_Hwi_enableInterrupt__E                  
80009c38  ti_sysbios_family_arm_a8_intcps_Hwi_getStackInfo__E                     
8000b6a4  ti_sysbios_family_arm_a8_intcps_Hwi_initVbar__I                         
8000b0f0  ti_sysbios_family_arm_a8_intcps_Hwi_init__I                             
48200000  ti_sysbios_family_arm_a8_intcps_Hwi_intc                                
8000a1a0  ti_sysbios_family_arm_a8_intcps_Hwi_nonPluggedHwiHandler__I             
8000b1bc  ti_sysbios_family_arm_a8_intcps_Hwi_startup__E                          
8000b56c  ti_sysbios_family_arm_a8_intcps_Hwi_switchFromBootStack__E              
8000fda8  ti_sysbios_family_arm_a8_intcps_Hwi_taskDisable__C                      
8000fdac  ti_sysbios_family_arm_a8_intcps_Hwi_taskRestoreHwi__C                   
80018400  ti_sysbios_family_arm_a8_intcps_Hwi_vectors                             
80017bd0  ti_sysbios_family_arm_a8_ti81xx_TimerSupport_Module_State_0_intNums__A  
8000afdc  ti_sysbios_family_arm_a8_ti81xx_TimerSupport_Module__startupDone__F     
8000afdc  ti_sysbios_family_arm_a8_ti81xx_TimerSupport_Module__startupDone__S     
80017bd8  ti_sysbios_family_arm_a8_ti81xx_TimerSupport_Module__state__V           
8000b784  ti_sysbios_family_arm_a8_ti81xx_TimerSupport_Module_startup__E          
8000b7cc  ti_sysbios_family_arm_a8_ti81xx_TimerSupport_enable__E                  
8000fdb0  ti_sysbios_family_arm_exc_Exception_E_dataAbort__C                      
8000fdb4  ti_sysbios_family_arm_exc_Exception_E_prefetchAbort__C                  
8000fdb8  ti_sysbios_family_arm_exc_Exception_E_swi__C                            
8000fdbc  ti_sysbios_family_arm_exc_Exception_E_undefinedInstruction__C           
80017bdc  ti_sysbios_family_arm_exc_Exception_Module_State_0_excActive__A         
80017be0  ti_sysbios_family_arm_exc_Exception_Module_State_0_excContext__A        
80017be4  ti_sysbios_family_arm_exc_Exception_Module_State_0_excStackBuffers__A   
8000b808  ti_sysbios_family_arm_exc_Exception_Module_State_0_excStack_0__A        
80017be8  ti_sysbios_family_arm_exc_Exception_Module_State_0_excStack__A          
8000ffbe  ti_sysbios_family_arm_exc_Exception_Module__id__C                       
80017bec  ti_sysbios_family_arm_exc_Exception_Module__state__V                    
8000b6b4  ti_sysbios_family_arm_exc_Exception_Module_startup__E                   
80004420  ti_sysbios_family_arm_exc_Exception_excDumpContext__I                   
800086a0  ti_sysbios_family_arm_exc_Exception_excHandlerAsm__I                    
80008708  ti_sysbios_family_arm_exc_Exception_excHandlerDataAsm__I                
80004f20  ti_sysbios_family_arm_exc_Exception_excHandler__I                       
8000fdc0  ti_sysbios_family_arm_exc_Exception_excHookFuncs__A                     
8000fdc4  ti_sysbios_family_arm_exc_Exception_excHookFuncs__C                     
80009ea8  ti_sysbios_family_arm_exc_Exception_initCore0__I                        
80009324  ti_sysbios_family_xxx_Hwi_switchAndRunFunc                              
800092e0  ti_sysbios_family_xxx_Hwi_switchToIsrStack                              
80009308  ti_sysbios_family_xxx_Hwi_switchToTaskStack                             
8000ae30  ti_sysbios_gates_GateHwi_Handle__label__S                               
8000b7d0  ti_sysbios_gates_GateHwi_Instance_init__E                               
8000fb2c  ti_sysbios_gates_GateHwi_Module__FXNS__C                                
80017c00  ti_sysbios_gates_GateHwi_Module__root__V                                
8000fbe0  ti_sysbios_gates_GateHwi_Object__DESC__C                                
8000fcdc  ti_sysbios_gates_GateHwi_Object__PARAMS__C                              
8000a450  ti_sysbios_gates_GateHwi_Object__create__S                              
8000ad10  ti_sysbios_gates_GateHwi_Object__delete__S                              
80017c08  ti_sysbios_gates_GateHwi_Object__table__V                               
8000b6c4  ti_sysbios_gates_GateHwi_enter__E                                       
8000b78c  ti_sysbios_gates_GateHwi_leave__E                                       
8000b794  ti_sysbios_gates_GateHwi_query__E                                       
8000fdc8  ti_sysbios_gates_GateMutex_A_badContext__C                              
8000ae5c  ti_sysbios_gates_GateMutex_Handle__label__S                             
8000fdcc  ti_sysbios_gates_GateMutex_Instance_State_sem__O                        
8000b580  ti_sysbios_gates_GateMutex_Instance_finalize__E                         
8000ad40  ti_sysbios_gates_GateMutex_Instance_init__E                             
8000fb50  ti_sysbios_gates_GateMutex_Module__FXNS__C                              
8000fdd0  ti_sysbios_gates_GateMutex_Module__diagsEnabled__C                      
8000fdd4  ti_sysbios_gates_GateMutex_Module__diagsIncluded__C                     
8000fdd8  ti_sysbios_gates_GateMutex_Module__diagsMask__C                         
8000ffc0  ti_sysbios_gates_GateMutex_Module__id__C                                
80017c0c  ti_sysbios_gates_GateMutex_Module__root__V                              
8000fc00  ti_sysbios_gates_GateMutex_Object__DESC__C                              
8000fcf4  ti_sysbios_gates_GateMutex_Object__PARAMS__C                            
8000a4a0  ti_sysbios_gates_GateMutex_Object__create__S                            
8000ab44  ti_sysbios_gates_GateMutex_Object__delete__S                            
80018144  ti_sysbios_gates_GateMutex_Object__table__V                             
80007828  ti_sysbios_gates_GateMutex_enter__E                                     
8000ae88  ti_sysbios_gates_GateMutex_leave__E                                     
8000b79c  ti_sysbios_gates_GateMutex_query__E                                     
80009e44  ti_sysbios_hal_Cache_CacheProxy_disable__E                              
8000a84c  ti_sysbios_hal_Cache_CacheProxy_enable__E                               
800091b8  ti_sysbios_hal_Cache_CacheProxy_wbInvAll__E                             
8000fddc  ti_sysbios_hal_Hwi_E_stackOverflow__C                                   
8000afb4  ti_sysbios_hal_Hwi_HwiProxy_Module__startupDone__S                      
8000b558  ti_sysbios_hal_Hwi_HwiProxy_clearInterrupt__E                           
8000805c  ti_sysbios_hal_Hwi_HwiProxy_disableInterrupt__E                         
8000814c  ti_sysbios_hal_Hwi_HwiProxy_enableInterrupt__E                          
80009c38  ti_sysbios_hal_Hwi_HwiProxy_getStackInfo__E                             
8000b1bc  ti_sysbios_hal_Hwi_HwiProxy_startup__E                                  
8000b56c  ti_sysbios_hal_Hwi_HwiProxy_switchFromBootStack__E                      
8000ffc2  ti_sysbios_hal_Hwi_Module__id__C                                        
80017c14  ti_sysbios_hal_Hwi_Module__root__V                                      
8000b438  ti_sysbios_hal_Hwi_Module_startup__E                                    
80017c1c  ti_sysbios_hal_Hwi_Object__table__V                                     
8000a1f8  ti_sysbios_hal_Hwi_checkStack                                           
8000a5dc  ti_sysbios_hal_Hwi_initStack                                            
8000fde0  ti_sysbios_heaps_HeapMem_A_align__C                                     
8000fde4  ti_sysbios_heaps_HeapMem_A_heapSize__C                                  
8000fde8  ti_sysbios_heaps_HeapMem_A_invalidFree__C                               
8000fdec  ti_sysbios_heaps_HeapMem_A_zeroBlock__C                                 
8000fdf0  ti_sysbios_heaps_HeapMem_E_memory__C                                    
8000aeb4  ti_sysbios_heaps_HeapMem_Handle__label__S                               
8000d808  ti_sysbios_heaps_HeapMem_Instance_State_0_buf__A                        
80005a5c  ti_sysbios_heaps_HeapMem_Instance_init__E                               
8000ae5c  ti_sysbios_heaps_HeapMem_Module_GateProxy_Handle__label__S              
8000ab44  ti_sysbios_heaps_HeapMem_Module_GateProxy_Object__delete__S             
8000b7d4  ti_sysbios_heaps_HeapMem_Module_GateProxy_enter__E                      
8000b7d8  ti_sysbios_heaps_HeapMem_Module_GateProxy_leave__E                      
8000b79c  ti_sysbios_heaps_HeapMem_Module_GateProxy_query__E                      
8000fb04  ti_sysbios_heaps_HeapMem_Module__FXNS__C                                
8000fdf4  ti_sysbios_heaps_HeapMem_Module__diagsEnabled__C                        
8000fdf8  ti_sysbios_heaps_HeapMem_Module__diagsIncluded__C                       
8000fdfc  ti_sysbios_heaps_HeapMem_Module__diagsMask__C                           
8000fe00  ti_sysbios_heaps_HeapMem_Module__gateObj__C                             
8000ffc4  ti_sysbios_heaps_HeapMem_Module__id__C                                  
80017c24  ti_sysbios_heaps_HeapMem_Module__root__V                                
8000fc20  ti_sysbios_heaps_HeapMem_Object__DESC__C                                
8000fb74  ti_sysbios_heaps_HeapMem_Object__PARAMS__C                              
8000fe04  ti_sysbios_heaps_HeapMem_Object__count__C                               
8000a4f0  ti_sysbios_heaps_HeapMem_Object__create__S                              
8000ad70  ti_sysbios_heaps_HeapMem_Object__delete__S                              
8000b2c4  ti_sysbios_heaps_HeapMem_Object__get__S                                 
80017c2c  ti_sysbios_heaps_HeapMem_Object__table__V                               
800036c4  ti_sysbios_heaps_HeapMem_alloc__E                                       
80003334  ti_sysbios_heaps_HeapMem_free__E                                        
80009698  ti_sysbios_heaps_HeapMem_getStats__E                                    
80009d0c  ti_sysbios_heaps_HeapMem_init__I                                        
8000b7a4  ti_sysbios_heaps_HeapMem_isBlocking__E                                  
8000fe08  ti_sysbios_heaps_HeapMem_reqAlign__C                                    
8000fe0c  ti_sysbios_knl_Clock_LM_begin__C                                        
8000fe10  ti_sysbios_knl_Clock_LM_tick__C                                         
8000fe14  ti_sysbios_knl_Clock_LW_delayed__C                                      
8000fe18  ti_sysbios_knl_Clock_Module_State_clockQ__O                             
8000fe1c  ti_sysbios_knl_Clock_Module__diagsEnabled__C                            
8000fe20  ti_sysbios_knl_Clock_Module__diagsIncluded__C                           
8000fe24  ti_sysbios_knl_Clock_Module__diagsMask__C                               
8000ffc6  ti_sysbios_knl_Clock_Module__id__C                                      
8000ffc8  ti_sysbios_knl_Clock_Module__loggerDefined__C                           
8000fe28  ti_sysbios_knl_Clock_Module__loggerFxn1__C                              
8000fe2c  ti_sysbios_knl_Clock_Module__loggerFxn2__C                              
8000fe30  ti_sysbios_knl_Clock_Module__loggerObj__C                               
80017c44  ti_sysbios_knl_Clock_Module__root__V                                    
80018210  ti_sysbios_knl_Clock_Module__state__V                                   
8000ab78  ti_sysbios_knl_Clock_Module_startup__E                                  
80017c4c  ti_sysbios_knl_Clock_Object__table__V                                   
8000b02c  ti_sysbios_knl_Clock_TimerProxy_Module__startupDone__S                  
8000b7dc  ti_sysbios_knl_Clock_TimerProxy_getMaxTicks__E                          
80009a70  ti_sysbios_knl_Clock_TimerProxy_startup__E                              
8000a6fc  ti_sysbios_knl_Clock_doTick__I                                          
80008cf4  ti_sysbios_knl_Clock_logTick__E                                         
80006010  ti_sysbios_knl_Clock_workFunc__E                                        
8000fe34  ti_sysbios_knl_Idle_funcList__A                                         
8000fd54  ti_sysbios_knl_Idle_funcList__C                                         
8000b720  ti_sysbios_knl_Idle_loop__E                                             
8000abac  ti_sysbios_knl_Idle_run__E                                              
8000b72c  ti_sysbios_knl_Queue_Instance_init__E                                   
80017c6c  ti_sysbios_knl_Queue_Module__root__V                                    
8000fc40  ti_sysbios_knl_Queue_Object__DESC__C                                    
8000fd0c  ti_sysbios_knl_Queue_Object__PARAMS__C                                  
8000b004  ti_sysbios_knl_Queue_Object__destruct__S                                
8000b6d4  ti_sysbios_knl_Queue_Object__get__S                                     
8000a628  ti_sysbios_knl_Queue_construct                                          
8000b7e0  ti_sysbios_knl_Queue_destruct                                           
8000b450  ti_sysbios_knl_Queue_empty__E                                           
8000fe38  ti_sysbios_knl_Semaphore_A_badContext__C                                
8000fe3c  ti_sysbios_knl_Semaphore_A_noEvents__C                                  
8000fe40  ti_sysbios_knl_Semaphore_A_overflow__C                                  
8000fe44  ti_sysbios_knl_Semaphore_A_pendTaskDisabled__C                          
8000fe48  ti_sysbios_knl_Semaphore_Instance_State_pendQ__O                        
8000b594  ti_sysbios_knl_Semaphore_Instance_finalize__E                           
80007a70  ti_sysbios_knl_Semaphore_Instance_init__E                               
8000fe4c  ti_sysbios_knl_Semaphore_LM_pend__C                                     
8000fe50  ti_sysbios_knl_Semaphore_LM_post__C                                     
8000fe54  ti_sysbios_knl_Semaphore_Module__diagsEnabled__C                        
8000fe58  ti_sysbios_knl_Semaphore_Module__diagsIncluded__C                       
8000fe5c  ti_sysbios_knl_Semaphore_Module__diagsMask__C                           
8000ffca  ti_sysbios_knl_Semaphore_Module__id__C                                  
8000ffcc  ti_sysbios_knl_Semaphore_Module__loggerDefined__C                       
8000fe60  ti_sysbios_knl_Semaphore_Module__loggerFxn2__C                          
8000fe64  ti_sysbios_knl_Semaphore_Module__loggerFxn4__C                          
8000fe68  ti_sysbios_knl_Semaphore_Module__loggerObj__C                           
80017c74  ti_sysbios_knl_Semaphore_Module__root__V                                
8000fc60  ti_sysbios_knl_Semaphore_Object__DESC__C                                
8000fb98  ti_sysbios_knl_Semaphore_Object__PARAMS__C                              
8000aee0  ti_sysbios_knl_Semaphore_Object__destruct__S                            
8000a540  ti_sysbios_knl_Semaphore_construct                                      
8000b7e4  ti_sysbios_knl_Semaphore_destruct                                       
8000a300  ti_sysbios_knl_Semaphore_pendTimeout__I                                 
80002e68  ti_sysbios_knl_Semaphore_pend__E                                        
80005c54  ti_sysbios_knl_Semaphore_post__E                                        
8000fe6c  ti_sysbios_knl_Swi_LD_end__C                                            
8000fe70  ti_sysbios_knl_Swi_LM_begin__C                                          
8000fe74  ti_sysbios_knl_Swi_LM_post__C                                           
80017eb8  ti_sysbios_knl_Swi_Module_State_0_readyQ__A                             
8000fe78  ti_sysbios_knl_Swi_Module__diagsEnabled__C                              
8000fe7c  ti_sysbios_knl_Swi_Module__diagsIncluded__C                             
8000fe80  ti_sysbios_knl_Swi_Module__diagsMask__C                                 
8000ffce  ti_sysbios_knl_Swi_Module__id__C                                        
8000ffd0  ti_sysbios_knl_Swi_Module__loggerDefined__C                             
8000fe84  ti_sysbios_knl_Swi_Module__loggerFxn1__C                                
8000fe88  ti_sysbios_knl_Swi_Module__loggerFxn4__C                                
8000fe8c  ti_sysbios_knl_Swi_Module__loggerObj__C                                 
80017c7c  ti_sysbios_knl_Swi_Module__root__V                                      
80017c84  ti_sysbios_knl_Swi_Module__state__V                                     
8000a984  ti_sysbios_knl_Swi_Module_startup__E                                    
8000fe90  ti_sysbios_knl_Swi_Object__count__C                                     
8000b2e0  ti_sysbios_knl_Swi_Object__get__S                                       
800181b0  ti_sysbios_knl_Swi_Object__table__V                                     
8000b468  ti_sysbios_knl_Swi_disable__E                                           
8000794c  ti_sysbios_knl_Swi_post__E                                              
80008d90  ti_sysbios_knl_Swi_restoreHwi__E                                        
80009718  ti_sysbios_knl_Swi_runLoop__I                                           
800061c8  ti_sysbios_knl_Swi_run__I                                               
80009590  ti_sysbios_knl_Swi_schedule__I                                          
8000a250  ti_sysbios_knl_Swi_startup__E                                           
8000fe94  ti_sysbios_knl_Task_A_badPriority__C                                    
8000fe98  ti_sysbios_knl_Task_A_badTaskState__C                                   
8000fe9c  ti_sysbios_knl_Task_A_badThreadType__C                                  
8000fea0  ti_sysbios_knl_Task_A_badTimeout__C                                     
8000fea4  ti_sysbios_knl_Task_A_noPendElem__C                                     
8000fea8  ti_sysbios_knl_Task_A_sleepTaskDisabled__C                              
8000feac  ti_sysbios_knl_Task_E_spOutOfBounds__C                                  
8000feb0  ti_sysbios_knl_Task_E_stackOverflow__C                                  
8000e808  ti_sysbios_knl_Task_Instance_State_0_stack__A                           
80003a40  ti_sysbios_knl_Task_Instance_finalize__E                                
8000471c  ti_sysbios_knl_Task_Instance_init__E                                    
8000feb4  ti_sysbios_knl_Task_LD_block__C                                         
8000feb8  ti_sysbios_knl_Task_LD_exit__C                                          
8000febc  ti_sysbios_knl_Task_LD_ready__C                                         
8000fec0  ti_sysbios_knl_Task_LM_sleep__C                                         
8000fec4  ti_sysbios_knl_Task_LM_switch__C                                        
80017ca8  ti_sysbios_knl_Task_Module_State_0_idleTask__A                          
80017f38  ti_sysbios_knl_Task_Module_State_0_readyQ__A                            
8000fec8  ti_sysbios_knl_Task_Module_State_inactiveQ__O                           
8000fecc  ti_sysbios_knl_Task_Module__diagsEnabled__C                             
8000fed0  ti_sysbios_knl_Task_Module__diagsIncluded__C                            
8000fed4  ti_sysbios_knl_Task_Module__diagsMask__C                                
8000ffd2  ti_sysbios_knl_Task_Module__id__C                                       
8000ffd4  ti_sysbios_knl_Task_Module__loggerDefined__C                            
8000fed8  ti_sysbios_knl_Task_Module__loggerFxn2__C                               
8000fedc  ti_sysbios_knl_Task_Module__loggerFxn4__C                               
8000fee0  ti_sysbios_knl_Task_Module__loggerObj__C                                
80017ca0  ti_sysbios_knl_Task_Module__root__V                                     
80018100  ti_sysbios_knl_Task_Module__state__V                                    
800051a0  ti_sysbios_knl_Task_Module_startup__E                                   
8000fc80  ti_sysbios_knl_Task_Object__DESC__C                                     
8000fa58  ti_sysbios_knl_Task_Object__PARAMS__C                                   
8000fee4  ti_sysbios_knl_Task_Object__count__C                                    
8000b480  ti_sysbios_knl_Task_Object__get__S                                      
8001806c  ti_sysbios_knl_Task_Object__table__V                                    
8000b75c  ti_sysbios_knl_Task_SupportProxy_Module__startupDone__S                 
8000b51c  ti_sysbios_knl_Task_SupportProxy_checkStack__E                          
8000b654  ti_sysbios_knl_Task_SupportProxy_getStackAlignment__E                   
80009ca4  ti_sysbios_knl_Task_SupportProxy_start__E                               
8000b3c0  ti_sysbios_knl_Task_SupportProxy_swap__E                                
8000fee8  ti_sysbios_knl_Task_allBlockedFunc__C                                   
80009614  ti_sysbios_knl_Task_allBlockedFunction__I                               
80007c7c  ti_sysbios_knl_Task_blockI__E                                           
8000749c  ti_sysbios_knl_Task_checkStacks__E                                      
80008e2c  ti_sysbios_knl_Task_create                                              
8000feec  ti_sysbios_knl_Task_defaultStackHeap__C                                 
8000fef0  ti_sysbios_knl_Task_defaultStackSize__C                                 
8000b498  ti_sysbios_knl_Task_disable__E                                          
8000abe0  ti_sysbios_knl_Task_enter__I                                            
80008328  ti_sysbios_knl_Task_exit__E                                             
8000ffd6  ti_sysbios_knl_Task_initStackFlag__C                                    
8000fef4  ti_sysbios_knl_Task_numConstructedTasks__C                              
80007b78  ti_sysbios_knl_Task_postInit__I                                         
8000a354  ti_sysbios_knl_Task_processVitalTaskFlag__I                             
8000a740  ti_sysbios_knl_Task_restoreHwi__E                                       
8000a030  ti_sysbios_knl_Task_restore__E                                          
800070e8  ti_sysbios_knl_Task_schedule__I                                         
8000b114  ti_sysbios_knl_Task_sleepTimeout__I                                     
800040fc  ti_sysbios_knl_Task_sleep__E                                            
80007224  ti_sysbios_knl_Task_startCore__E                                        
8000b7e8  ti_sysbios_knl_Task_startup__E                                          
80007d78  ti_sysbios_knl_Task_unblockI__E                                         
8000fef8  ti_sysbios_timers_dmtimer_Timer_E_cannotSupport__C                      
8000fefc  ti_sysbios_timers_dmtimer_Timer_E_freqMismatch__C                       
800180b8  ti_sysbios_timers_dmtimer_Timer_Module_State_0_device__A                
80017cb4  ti_sysbios_timers_dmtimer_Timer_Module_State_0_handles__A               
800181e0  ti_sysbios_timers_dmtimer_Timer_Module_State_0_intFreqs__A              
8000ff00  ti_sysbios_timers_dmtimer_Timer_Module__diagsEnabled__C                 
8000ff04  ti_sysbios_timers_dmtimer_Timer_Module__diagsIncluded__C                
8000ff08  ti_sysbios_timers_dmtimer_Timer_Module__diagsMask__C                    
8000ffd8  ti_sysbios_timers_dmtimer_Timer_Module__id__C                           
80017cac  ti_sysbios_timers_dmtimer_Timer_Module__root__V                         
8000b02c  ti_sysbios_timers_dmtimer_Timer_Module__startupDone__F                  
8000b02c  ti_sysbios_timers_dmtimer_Timer_Module__startupDone__S                  
80017ccc  ti_sysbios_timers_dmtimer_Timer_Module__state__V                        
800088fc  ti_sysbios_timers_dmtimer_Timer_Module_startup__E                       
80017fb8  ti_sysbios_timers_dmtimer_Timer_Object__table__V                        
8000afdc  ti_sysbios_timers_dmtimer_Timer_TimerSupportProxy_Module__startupDone__S
8000b7cc  ti_sysbios_timers_dmtimer_Timer_TimerSupportProxy_enable__E             
80005638  ti_sysbios_timers_dmtimer_Timer_checkFreq__I                            
8000ffda  ti_sysbios_timers_dmtimer_Timer_checkFrequency__C                       
80006378  ti_sysbios_timers_dmtimer_Timer_deviceConfig__I                         
8000b738  ti_sysbios_timers_dmtimer_Timer_getMaxTicks__E                          
8000924c  ti_sysbios_timers_dmtimer_Timer_initDevice__I                           
8000ff0c  ti_sysbios_timers_dmtimer_Timer_numTimerDevices__C                      
80007360  ti_sysbios_timers_dmtimer_Timer_setPeriodMicroSecs__E                   
80008414  ti_sysbios_timers_dmtimer_Timer_start__E                                
8000ffdc  ti_sysbios_timers_dmtimer_Timer_startupNeeded__C                        
80009a70  ti_sysbios_timers_dmtimer_Timer_startup__E                              
80009f70  ti_sysbios_timers_dmtimer_Timer_stop__E                                 
8000a9c0  ti_sysbios_timers_dmtimer_Timer_stub__E                                 
8000ff10  xdc_runtime_Assert_E_assertFailed__C                                    
80009894  xdc_runtime_Assert_raise__I                                             
8000ff14  xdc_runtime_Core_A_initializedParams__C                                 
8000ff18  xdc_runtime_Core_Module__diagsEnabled__C                                
8000ff1c  xdc_runtime_Core_Module__diagsIncluded__C                               
8000ff20  xdc_runtime_Core_Module__diagsMask__C                                   
8000ffde  xdc_runtime_Core_Module__id__C                                          
8000a08c  xdc_runtime_Core_assignLabel__I                                         
80009f0c  xdc_runtime_Core_assignParams__I                                        
80006fa4  xdc_runtime_Core_constructObject__I                                     
800066d0  xdc_runtime_Core_createObject__I                                        
80008ec4  xdc_runtime_Core_deleteObject__I                                        
8000ff24  xdc_runtime_Error_E_memory__C                                           
8000ff28  xdc_runtime_Error_Module__diagsEnabled__C                               
8000ff2c  xdc_runtime_Error_Module__diagsIncluded__C                              
8000ff30  xdc_runtime_Error_Module__diagsMask__C                                  
8000ffe0  xdc_runtime_Error_Module__loggerDefined__C                              
8000ff34  xdc_runtime_Error_Module__loggerFxn8__C                                 
8000ff38  xdc_runtime_Error_Module__loggerObj__C                                  
80017ce0  xdc_runtime_Error_Module__state__V                                      
8000af0c  xdc_runtime_Error_check__E                                              
8000b7ac  xdc_runtime_Error_getSite__E                                            
8000b4b0  xdc_runtime_Error_init__E                                               
8000ffe2  xdc_runtime_Error_maxDepth__C                                           
80006528  xdc_runtime_Error_policyDefault__E                                      
8000ff3c  xdc_runtime_Error_policyFxn__C                                          
8000fd35  xdc_runtime_Error_policy__C                                             
80008f5c  xdc_runtime_Error_print__E                                              
8000ff40  xdc_runtime_Error_raiseHook__C                                          
8000ada0  xdc_runtime_Error_raiseX__E                                             
80009d74  xdc_runtime_Error_setX__E                                               
8000b6e4  xdc_runtime_Gate_enterSystem__E                                         
8000b5a8  xdc_runtime_Gate_leaveSystem__E                                         
8000ff44  xdc_runtime_IFilterLogger_Interface__BASE__C                            
8000ff48  xdc_runtime_IGateProvider_Interface__BASE__C                            
8000ff4c  xdc_runtime_IHeap_Interface__BASE__C                                    
8000ff50  xdc_runtime_ILogger_Interface__BASE__C                                  
8000ff54  xdc_runtime_IModule_Interface__BASE__C                                  
8000ff58  xdc_runtime_Log_L_error__C                                              
8000ff5c  xdc_runtime_LoggerBuf_E_badLevel__C                                     
8000af38  xdc_runtime_LoggerBuf_Handle__label__S                                  
8000f408  xdc_runtime_LoggerBuf_Instance_State_0_entryArr__A                      
8000b1dc  xdc_runtime_LoggerBuf_Instance_finalize__E                              
80009ddc  xdc_runtime_LoggerBuf_Instance_init__E                                  
8000ae30  xdc_runtime_LoggerBuf_Module_GateProxy_Handle__label__S                 
8000ad10  xdc_runtime_LoggerBuf_Module_GateProxy_Object__delete__S                
8000b7ec  xdc_runtime_LoggerBuf_Module_GateProxy_enter__E                         
8000b7f0  xdc_runtime_LoggerBuf_Module_GateProxy_leave__E                         
8000b794  xdc_runtime_LoggerBuf_Module_GateProxy_query__E                         
8000fa94  xdc_runtime_LoggerBuf_Module__FXNS__C                                   
8000ff60  xdc_runtime_LoggerBuf_Module__gateObj__C                                
8000ffe4  xdc_runtime_LoggerBuf_Module__id__C                                     
80017ce4  xdc_runtime_LoggerBuf_Module__root__V                                   
80017cec  xdc_runtime_LoggerBuf_Module__state__V                                  
8000a88c  xdc_runtime_LoggerBuf_Module_startup__E                                 
8000fca0  xdc_runtime_LoggerBuf_Object__DESC__C                                   
8000fbbc  xdc_runtime_LoggerBuf_Object__PARAMS__C                                 
8000ff64  xdc_runtime_LoggerBuf_Object__count__C                                  
80008ff4  xdc_runtime_LoggerBuf_Object__create__S                                 
8000ac14  xdc_runtime_LoggerBuf_Object__delete__S                                 
8000b2fc  xdc_runtime_LoggerBuf_Object__get__S                                    
80018260  xdc_runtime_LoggerBuf_Object__table__V                                  
8000b77c  xdc_runtime_LoggerBuf_TimestampProxy_get32__E                           
8000a590  xdc_runtime_LoggerBuf_TimestampProxy_get64__E                           
8000b644  xdc_runtime_LoggerBuf_TimestampProxy_getFreq__E                         
8000b5e4  xdc_runtime_LoggerBuf_disable__E                                        
8000b5f8  xdc_runtime_LoggerBuf_enable__E                                         
8000ffe6  xdc_runtime_LoggerBuf_filterByLevel__C                                  
80009ae4  xdc_runtime_LoggerBuf_filterOutEvent__I                                 
80008770  xdc_runtime_LoggerBuf_getFilterLevel__E                                 
8000aa70  xdc_runtime_LoggerBuf_reset__E                                          
800084f0  xdc_runtime_LoggerBuf_setFilterLevel__E                                 
8000ff68  xdc_runtime_LoggerBuf_statusLogger__C                                   
8000b318  xdc_runtime_LoggerBuf_write0__E                                         
8000b334  xdc_runtime_LoggerBuf_write1__E                                         
8000b1fc  xdc_runtime_LoggerBuf_write2__E                                         
800075d0  xdc_runtime_LoggerBuf_write4__E                                         
80005e38  xdc_runtime_LoggerBuf_write8__E                                         
8000ae30  xdc_runtime_Main_Module_GateProxy_Handle__label__S                      
8000ad10  xdc_runtime_Main_Module_GateProxy_Object__delete__S                     
8000b794  xdc_runtime_Main_Module_GateProxy_query__E                              
8000aeb4  xdc_runtime_Memory_HeapProxy_Handle__label__S                           
8000ad70  xdc_runtime_Memory_HeapProxy_Object__delete__S                          
8000b5bc  xdc_runtime_Memory_HeapProxy_alloc__E                                   
8000b5d0  xdc_runtime_Memory_HeapProxy_free__E                                    
8000ffe8  xdc_runtime_Memory_Module__id__C                                        
80017cf4  xdc_runtime_Memory_Module__state__V                                     
80008a60  xdc_runtime_Memory_alloc__E                                             
8000b60c  xdc_runtime_Memory_calloc__E                                            
8000ff6c  xdc_runtime_Memory_defaultHeapInstance__C                               
8000b620  xdc_runtime_Memory_free__E                                              
8000b6f4  xdc_runtime_Memory_getMaxDefaultTypeAlign__E                            
8000add0  xdc_runtime_Memory_valloc__E                                            
80017cf8  xdc_runtime_Registry_Module__state__V                                   
8000ac48  xdc_runtime_Registry_findById__E                                        
80017d00  xdc_runtime_Startup_Module__state__V                                    
00000001  xdc_runtime_Startup__EXECFXN__C                                         
00000001  xdc_runtime_Startup__RESETFXN__C                                        
8000ff70  xdc_runtime_Startup_execImpl__C                                         
800093f8  xdc_runtime_Startup_exec__E                                             
8000b350  xdc_runtime_Startup_exec__I                                             
8000fd48  xdc_runtime_Startup_firstFxns__A                                        
8000fd5c  xdc_runtime_Startup_firstFxns__C                                        
8000fd64  xdc_runtime_Startup_lastFxns__C                                         
8000ff74  xdc_runtime_Startup_maxPasses__C                                        
8000b6a4  xdc_runtime_Startup_reset__I                                            
8000b704  xdc_runtime_Startup_rtsDone__E                                          
8000fcc0  xdc_runtime_Startup_sfxnRts__A                                          
8000ff78  xdc_runtime_Startup_sfxnRts__C                                          
8000fad0  xdc_runtime_Startup_sfxnTab__A                                          
8000ff7c  xdc_runtime_Startup_sfxnTab__C                                          
80006e50  xdc_runtime_Startup_startMods__I                                        
8000f608  xdc_runtime_SysMin_Module_State_0_outbuf__A                             
80017d08  xdc_runtime_SysMin_Module__state__V                                     
8000ac7c  xdc_runtime_SysMin_Module_startup__E                                    
8000a2a8  xdc_runtime_SysMin_abort__E                                             
8000ff80  xdc_runtime_SysMin_bufSize__C                                           
8000ae00  xdc_runtime_SysMin_exit__E                                              
8000ffea  xdc_runtime_SysMin_flushAtExit__C                                       
80009bc8  xdc_runtime_SysMin_flush__E                                             
8000ff84  xdc_runtime_SysMin_outputFunc__C                                        
8000a784  xdc_runtime_SysMin_output__I                                            
8000a0e8  xdc_runtime_SysMin_putch__E                                             
8000b36c  xdc_runtime_SysMin_ready__E                                             
8000ae30  xdc_runtime_System_Module_GateProxy_Handle__label__S                    
8000ad10  xdc_runtime_System_Module_GateProxy_Object__delete__S                   
8000b7f4  xdc_runtime_System_Module_GateProxy_enter__E                            
8000b7f8  xdc_runtime_System_Module_GateProxy_leave__E                            
8000b794  xdc_runtime_System_Module_GateProxy_query__E                            
80017d14  xdc_runtime_System_Module_State_0_atexitHandlers__A                     
8000ff88  xdc_runtime_System_Module__gateObj__C                                   
80017d24  xdc_runtime_System_Module__state__V                                     
8000b7b4  xdc_runtime_System_Module_startup__E                                    
8000a2a8  xdc_runtime_System_SupportProxy_abort__E                                
8000ae00  xdc_runtime_System_SupportProxy_exit__E                                 
80009bc8  xdc_runtime_System_SupportProxy_flush__E                                
8000a0e8  xdc_runtime_System_SupportProxy_putch__E                                
8000b36c  xdc_runtime_System_SupportProxy_ready__E                                
8000ff8c  xdc_runtime_System_abortFxn__C                                          
80009918  xdc_runtime_System_abortStd__E                                          
8000b054  xdc_runtime_System_abort__E                                             
8000b07c  xdc_runtime_System_aprintf__E                                           
8000b7fc  xdc_runtime_System_aprintf_va__F                                        
8000a144  xdc_runtime_System_atexit__E                                            
8000a8cc  xdc_runtime_System_avprintf__E                                          
80002468  xdc_runtime_System_doPrint__I                                           
8000ff90  xdc_runtime_System_exitFxn__C                                           
80009924  xdc_runtime_System_exitStd__E                                           
8000b138  xdc_runtime_System_exit__E                                              
8000ff94  xdc_runtime_System_extendFxn__C                                         
8000908c  xdc_runtime_System_formatNum__I                                         
8000ff98  xdc_runtime_System_maxAtexitHandlers__C                                 
80006874  xdc_runtime_System_printfExtend__I                                      
8000b0a4  xdc_runtime_System_printf__E                                            
8000b800  xdc_runtime_System_printf_va__F                                         
8000a670  xdc_runtime_System_processAtExit__E                                     
8000a3a8  xdc_runtime_System_putchar__I                                           
8000a9fc  xdc_runtime_System_vprintf__E                                           
8000b388  xdc_runtime_System_vsnprintf__E                                         
80017d2c  xdc_runtime_Text_Module__state__V                                       
8000ffec  xdc_runtime_Text_charCnt__C                                             
80014000  xdc_runtime_Text_charTab__A                                             
8000ff9c  xdc_runtime_Text_charTab__C                                             
8000a7c8  xdc_runtime_Text_cordText__E                                            
8000ffee  xdc_runtime_Text_isLoaded__C                                            
8000ffa0  xdc_runtime_Text_nameEmpty__C                                           
8000ffa4  xdc_runtime_Text_nameStatic__C                                          
8000ffa8  xdc_runtime_Text_nameUnknown__C                                         
8000f930  xdc_runtime_Text_nodeTab__A                                             
8000ffac  xdc_runtime_Text_nodeTab__C                                             
8000a3fc  xdc_runtime_Text_printVisFxn__I                                         
80008c54  xdc_runtime_Text_putLab__E                                              
800085c8  xdc_runtime_Text_putMod__E                                              
80007f68  xdc_runtime_Text_putSite__E                                             
8000fff0  xdc_runtime_Text_registryModsLastId__C                                  
8000b3a4  xdc_runtime_Text_ropeText__E                                            
8000fff2  xdc_runtime_Text_unnamedModsLastId__C                                   
80009798  xdc_runtime_Text_visitRope2__I                                          
8000ffb0  xdc_runtime_Text_visitRopeFxn__C                                        
8000b4c8  xdc_runtime_Text_visitRope__I                                           
80009fd0  xdc_runtime_Text_xprintf__I                                             
8000b77c  xdc_runtime_Timestamp_SupportProxy_get32__E                             
8000a590  xdc_runtime_Timestamp_SupportProxy_get64__E                             
8000b644  xdc_runtime_Timestamp_SupportProxy_getFreq__E                           


GLOBAL SYMBOLS: SORTED BY Symbol Address 

address   name                                                                    
-------   ----                                                                    
00000000  _argsize                                                                
00000001  xdc_runtime_Startup__EXECFXN__C                                         
00000001  xdc_runtime_Startup__RESETFXN__C                                        
00002000  __STACK_SIZE                                                            
48200000  ti_sysbios_family_arm_a8_intcps_Hwi_intc                                
80000000  GPMCRevisionGet                                                         
80000000  __ASM__                                                                 
80000024  GPMCIdleModeSelect                                                      
8000005c  __ISA__                                                                 
8000006c  GPMCAutoIdleConfig                                                      
8000006e  __PLAT__                                                                
80000094  __TARG__                                                                
800000a4  GPMCModuleSoftReset                                                     
800000bc  __TRDR__                                                                
800000c0  GPMCModuleResetStatusGet                                                
800000e4  GPMCIntStatusGet                                                        
80000188  GPMCIntStatusClear                                                      
80000228  GPMCIntEnable                                                           
800002c8  GPMCIntDisable                                                          
80000368  GPMCTimeOutStartValSet                                                  
800003b0  GPMCTimeOutFeatureConfig                                                
80000408  GPMCErrAddrGet                                                          
8000042c  GPMCErrValStatusGet                                                     
80000450  GPMCErrSysCmdGet                                                        
80000478  GPMCErrStatusGet                                                        
80000500  GPMCWaitPinPolaritySelect                                               
800005bc  GPMCWriteProtectPinLevelCtrl                                            
80000614  GPMCLimitedAddrDevSupportConfig                                         
8000066c  GPMCNANDForcePostedWriteFeatureConfig                                   
800006c4  GPMCWaitPinStatusGet                                                    
80000728  GPMCEmptyWriteBuffStatusGet                                             
8000074c  GPMCFclkDividerSelect                                                   
800007b4  GPMCTimeParaGranularitySelect                                           
80000820  GPMCAddrDataMuxProtocolSelect                                           
8000088c  GPMCDevTypeSelect                                                       
800008f8  GPMCDevSizeSelect                                                       
80000964  GPMCWaitPinSelect                                                       
800009d0  GPMCWaitMonitoringTimeSelect                                            
80000a3c  GPMCWaitPinMonitoringConfig                                             
80000b1c  GPMCClkActivationTimeConfig                                             
80000b88  GPMCDevPageLenSet                                                       
80000bf4  GPMCWriteTypeSelect                                                     
80000c60  GPMCReadTypeSelect                                                      
80000ccc  GPMCAccessTypeSelect                                                    
80000dac  GPMCSyncWrapBurstConfig                                                 
80000e18  GPMCCSTimingConfig                                                      
80000e4c  GPMCADVTimingConfig                                                     
80000e80  GPMCWEAndOETimingConfig                                                 
80000eb4  GPMCRdAccessAndCycleTimeTimingConfig                                    
80000ee8  GPMCWrAccessAndWrDataOnADMUXBusTimingConfig                             
80000f4c  GPMCycle2CycleAndTurnArndTimeTimingConfig                               
80000f8c  GPMCCSConfig                                                            
80000ff8  GPMCBaseAddrSet                                                         
80001060  GPMCMaskAddrSet                                                         
800010cc  GPMCSNANDCmdWrite                                                       
80001100  GPMCNANDAddrWrite                                                       
80001134  GPMCNANDDataWrite                                                       
80001168  GPMCNANDDataRead                                                        
8000119c  GPMCPrefetchAccessModeSelect                                            
800011e0  GPMCPrefetchSyncTypeSelect                                              
80001228  GPMCPrefetchSyncModeConfig                                              
80001270  GPMCPrefetchWaitPinSelect                                               
800012b8  GPMCPrefetchEngineEnable                                                
800012dc  GPMCPrefetchEngineDisable                                               
80001300  GPMCPrefetchFifoThrldValSet                                             
80001348  GPMCPrefetchCSSelect                                                    
80001390  GPMCPrefetchAccessCycleOptConfig                                        
800013d8  GPMCPrefetchCycleOptValSet                                              
80001420  GPMCPrefetchRRArbitrationConfig                                         
80001468  GPMCPrefetchWeightedPrioSet                                             
800014b0  GPMCPrefetchTrnsCntValSet                                               
800014f4  GPMCPrefetchEngineStart                                                 
80001510  GPMCPrefetchEngineStop                                                  
8000152c  GPMCPrefetchEngineStatusGet                                             
80001550  GPMCPrefetchCountValGet                                                 
80001574  GPMCPrefetchFifoThrldStatusGet                                          
8000159c  GPMCPrefetchFifoPtrValGet                                               
800015c4  GPMCECCAlgoSelect                                                       
8000160c  GPMCECCBCHErrCorrectionCapSelect                                        
80001654  GPMCECCBCHWrapModeValSet                                                
8000169c  GPMCECCColumnSelect                                                     
800016e4  GPMCECCBCHNumOfSectorsSelect                                            
8000172c  GPMCECCCSSelect                                                         
80001774  GPMCECCEnable                                                           
80001798  GPMCECCDisable                                                          
800017bc  GPMCECCResultRegClear                                                   
800017e0  GPMCECCResultRegSelect                                                  
80001824  GPMCECCSizeValSet                                                       
800018c0  GPMCECCResultSizeSelect                                                 
80001b0c  GPMCECCResultGet                                                        
80001b38  GPMCECCBCHResultGet                                                     
80001c44  GPMCECCBCHSWDataWrite                                                   
80001c68  GPMCECCBCHSWDataRead                                                    
80001c8c  GPMCSystemConfig                                                        
80001cac  GPMCMuxConfig1                                                          
80001dc4  GPMCMuxConfig2                                                          
80001e40  GPMCMuxConfig3                                                          
80001f04  GPMCMuxConfig4                                                          
80001fe0  GPMCMuxConfig5                                                          
8000205c  GPMCMuxConfig6                                                          
800020fc  GPMCMuxConfig7                                                          
8000213c  GpmcInitial                                                             
80002200  GpmcWriteFpga                                                           
80002268  GpmcReadFpga                                                            
80002468  xdc_runtime_System_doPrint__I                                           
8000299c  HOSTwrite                                                               
80002a20  HOSTunlink                                                              
80002a84  HOSTtime                                                                
80002ae4  HOSTrename                                                              
80002b7c  HOSTread                                                                
80002c00  HOSTopen                                                                
80002c8c  HOSTlseek                                                               
80002d2c  HOSTgetenv                                                              
80002d94  HOSTclose                                                               
80002dfc  HOSTclock                                                               
80002e68  ti_sysbios_knl_Semaphore_pend__E                                        
80003334  ti_sysbios_heaps_HeapMem_free__E                                        
800036c4  ti_sysbios_heaps_HeapMem_alloc__E                                       
80003a40  ti_sysbios_knl_Task_Instance_finalize__E                                
80003db8  ti_sysbios_family_arm_a8_Mmu_initTableBuf__I                            
800040fc  ti_sysbios_knl_Task_sleep__E                                            
80004420  ti_sysbios_family_arm_exc_Exception_excDumpContext__I                   
8000471c  ti_sysbios_knl_Task_Instance_init__E                                    
800049dc  __aeabi_uldivmod                                                        
80004c94  ti_sysbios_family_arm_a8_Mmu_setFirstLevelDesc__E                       
80004f20  ti_sysbios_family_arm_exc_Exception_excHandler__I                       
800051a0  ti_sysbios_knl_Task_Module_startup__E                                   
80005400  taskFxn                                                                 
80005450  main                                                                    
80005638  ti_sysbios_timers_dmtimer_Timer_checkFreq__I                            
80005860  ti_sysbios_family_arm_a8_intcps_Hwi_dispatchIRQC__I                     
80005a5c  ti_sysbios_heaps_HeapMem_Instance_init__E                               
80005c54  ti_sysbios_knl_Semaphore_post__E                                        
80005e38  xdc_runtime_LoggerBuf_write8__E                                         
80006010  ti_sysbios_knl_Clock_workFunc__E                                        
800061c8  ti_sysbios_knl_Swi_run__I                                               
80006378  ti_sysbios_timers_dmtimer_Timer_deviceConfig__I                         
80006528  xdc_runtime_Error_policyDefault__E                                      
800066d0  xdc_runtime_Core_createObject__I                                        
80006874  xdc_runtime_System_printfExtend__I                                      
800069fc  __aeabi_memcpy                                                          
800069fc  __aeabi_memcpy4                                                         
800069fc  __aeabi_memcpy8                                                         
800069fc  memcpy                                                                  
80006b7c  ti_sysbios_family_arm_a8_Cache_startup__I                               
80006cf4  ti_sysbios_family_arm_a8_intcps_Hwi_Module_startup__E                   
80006e50  xdc_runtime_Startup_startMods__I                                        
80006fa4  xdc_runtime_Core_constructObject__I                                     
800070e8  ti_sysbios_knl_Task_schedule__I                                         
80007224  ti_sysbios_knl_Task_startCore__E                                        
80007360  ti_sysbios_timers_dmtimer_Timer_setPeriodMicroSecs__E                   
8000749c  ti_sysbios_knl_Task_checkStacks__E                                      
800075d0  xdc_runtime_LoggerBuf_write4__E                                         
80007704  ti_sysbios_family_arm_a8_Mmu_initDescAttrs__E                           
80007828  ti_sysbios_gates_GateMutex_enter__E                                     
8000794c  ti_sysbios_knl_Swi_post__E                                              
80007a70  ti_sysbios_knl_Semaphore_Instance_init__E                               
80007b78  ti_sysbios_knl_Task_postInit__I                                         
80007c7c  ti_sysbios_knl_Task_blockI__E                                           
80007d78  ti_sysbios_knl_Task_unblockI__E                                         
80007e74  __aeabi_uidiv                                                           
80007e74  __aeabi_uidivmod                                                        
80007f68  xdc_runtime_Text_putSite__E                                             
8000805c  ti_sysbios_family_arm_a8_intcps_Hwi_disableInterrupt__E                 
8000805c  ti_sysbios_hal_Hwi_HwiProxy_disableInterrupt__E                         
8000814c  ti_sysbios_family_arm_a8_intcps_Hwi_enableInterrupt__E                  
8000814c  ti_sysbios_hal_Hwi_HwiProxy_enableInterrupt__E                          
8000823c  __TI_auto_init                                                          
80008328  ti_sysbios_knl_Task_exit__E                                             
80008414  ti_sysbios_timers_dmtimer_Timer_start__E                                
800084f0  xdc_runtime_LoggerBuf_setFilterLevel__E                                 
800085c8  xdc_runtime_Text_putMod__E                                              
800086a0  ti_sysbios_family_arm_exc_Exception_excHandlerAsm__I                    
80008708  ti_sysbios_family_arm_exc_Exception_excHandlerDataAsm__I                
80008770  xdc_runtime_LoggerBuf_getFilterLevel__E                                 
8000883c  ti_sysbios_family_arm_a8_intcps_Hwi_dispatchIRQ__I                      
800088fc  ti_sysbios_timers_dmtimer_Timer_Module_startup__E                       
800089b0  __aeabi_memclr                                                          
800089b0  __aeabi_memclr4                                                         
800089b0  __aeabi_memclr8                                                         
800089b4  __aeabi_memset                                                          
800089b4  __aeabi_memset4                                                         
800089b4  __aeabi_memset8                                                         
800089c0  memset                                                                  
80008a60  xdc_runtime_Memory_alloc__E                                             
80008b10  __TI_writemsg                                                           
80008b58  C$$IO$$                                                                 
80008b60  __TI_readmsg                                                            
80008c54  xdc_runtime_Text_putLab__E                                              
80008cf4  ti_sysbios_knl_Clock_logTick__E                                         
80008d90  ti_sysbios_knl_Swi_restoreHwi__E                                        
80008e2c  ti_sysbios_knl_Task_create                                              
80008ec4  xdc_runtime_Core_deleteObject__I                                        
80008f5c  xdc_runtime_Error_print__E                                              
80008ff4  xdc_runtime_LoggerBuf_Object__create__S                                 
8000908c  xdc_runtime_System_formatNum__I                                         
80009124  ti_sysbios_family_arm_a8_Cache_invL1dAll__E                             
800091b8  ti_sysbios_family_arm_a8_Cache_wbInvAll__E                              
800091b8  ti_sysbios_hal_Cache_CacheProxy_wbInvAll__E                             
8000924c  ti_sysbios_timers_dmtimer_Timer_initDevice__I                           
800092e0  ti_sysbios_family_xxx_Hwi_switchToIsrStack                              
80009308  ti_sysbios_family_xxx_Hwi_switchToTaskStack                             
80009324  ti_sysbios_family_xxx_Hwi_switchAndRunFunc                              
8000936d  MMUInit                                                                 
800093f8  xdc_runtime_Startup_exec__E                                             
80009484  ti_sysbios_family_arm_a8_Mmu_Module_startup__E                          
8000950c  copy_in                                                                 
80009590  ti_sysbios_knl_Swi_schedule__I                                          
80009614  ti_sysbios_knl_Task_allBlockedFunction__I                               
80009698  ti_sysbios_heaps_HeapMem_getStats__E                                    
80009718  ti_sysbios_knl_Swi_runLoop__I                                           
80009798  xdc_runtime_Text_visitRope2__I                                          
80009818  ti_sysbios_family_arm_TaskSupport_buildTaskStack                        
80009894  xdc_runtime_Assert_raise__I                                             
80009910  C$$EXIT                                                                 
80009918  abort                                                                   
80009918  xdc_runtime_System_abortStd__E                                          
80009924  exit                                                                    
80009924  xdc_runtime_System_exitStd__E                                           
80009988  _c_int00                                                                
800099fc  ti_sysbios_family_arm_a8_intcps_Hwi_dispatchFIQC__I                     
80009a70  ti_sysbios_knl_Clock_TimerProxy_startup__E                              
80009a70  ti_sysbios_timers_dmtimer_Timer_startup__E                              
80009ae4  xdc_runtime_LoggerBuf_filterOutEvent__I                                 
80009b58  ti_sysbios_family_arm_a8_Mmu_enable__E                                  
80009bc8  xdc_runtime_SysMin_flush__E                                             
80009bc8  xdc_runtime_System_SupportProxy_flush__E                                
80009c38  ti_sysbios_family_arm_a8_intcps_Hwi_getStackInfo__E                     
80009c38  ti_sysbios_hal_Hwi_HwiProxy_getStackInfo__E                             
80009ca4  ti_sysbios_family_arm_TaskSupport_start__E                              
80009ca4  ti_sysbios_knl_Task_SupportProxy_start__E                               
80009d0c  ti_sysbios_heaps_HeapMem_init__I                                        
80009d74  xdc_runtime_Error_setX__E                                               
80009ddc  xdc_runtime_LoggerBuf_Instance_init__E                                  
80009e44  ti_sysbios_family_arm_a8_Cache_disable__E                               
80009e44  ti_sysbios_hal_Cache_CacheProxy_disable__E                              
80009ea8  ti_sysbios_family_arm_exc_Exception_initCore0__I                        
80009f0c  xdc_runtime_Core_assignParams__I                                        
80009f70  ti_sysbios_timers_dmtimer_Timer_stop__E                                 
80009fd0  xdc_runtime_Text_xprintf__I                                             
8000a030  ti_sysbios_knl_Task_restore__E                                          
8000a08c  xdc_runtime_Core_assignLabel__I                                         
8000a0e8  xdc_runtime_SysMin_putch__E                                             
8000a0e8  xdc_runtime_System_SupportProxy_putch__E                                
8000a144  xdc_runtime_System_atexit__E                                            
8000a1a0  ti_sysbios_family_arm_a8_intcps_Hwi_nonPluggedHwiHandler__I             
8000a1f8  ti_sysbios_hal_Hwi_checkStack                                           
8000a250  ti_sysbios_knl_Swi_startup__E                                           
8000a2a8  xdc_runtime_SysMin_abort__E                                             
8000a2a8  xdc_runtime_System_SupportProxy_abort__E                                
8000a300  ti_sysbios_knl_Semaphore_pendTimeout__I                                 
8000a354  ti_sysbios_knl_Task_processVitalTaskFlag__I                             
8000a3a8  xdc_runtime_System_putchar__I                                           
8000a3fc  xdc_runtime_Text_printVisFxn__I                                         
8000a450  ti_sysbios_gates_GateHwi_Object__create__S                              
8000a4a0  ti_sysbios_gates_GateMutex_Object__create__S                            
8000a4f0  ti_sysbios_heaps_HeapMem_Object__create__S                              
8000a540  ti_sysbios_knl_Semaphore_construct                                      
8000a590  ti_sysbios_family_arm_a8_TimestampProvider_get64__E                     
8000a590  xdc_runtime_LoggerBuf_TimestampProxy_get64__E                           
8000a590  xdc_runtime_Timestamp_SupportProxy_get64__E                             
8000a5dc  ti_sysbios_hal_Hwi_initStack                                            
8000a628  ti_sysbios_knl_Queue_construct                                          
8000a670  xdc_runtime_System_processAtExit__E                                     
8000a6b8  ti_sysbios_BIOS_atExitFunc__I                                           
8000a6fc  ti_sysbios_knl_Clock_doTick__I                                          
8000a740  ti_sysbios_knl_Task_restoreHwi__E                                       
8000a784  xdc_runtime_SysMin_output__I                                            
8000a7c8  xdc_runtime_Text_cordText__E                                            
8000a80d  PinMuxConfig                                                            
8000a83d  PRUSSPinMuxConfig                                                       
8000a84c  ti_sysbios_family_arm_a8_Cache_enable__E                                
8000a84c  ti_sysbios_hal_Cache_CacheProxy_enable__E                               
8000a88c  xdc_runtime_LoggerBuf_Module_startup__E                                 
8000a8cc  xdc_runtime_System_avprintf__E                                          
8000a90c  ti_sysbios_family_arm_a8_Mmu_disable__E                                 
8000a948  ti_sysbios_family_arm_a8_TimestampProvider_autoRefreshFxn__I            
8000a984  ti_sysbios_knl_Swi_Module_startup__E                                    
8000a9c0  ti_sysbios_timers_dmtimer_Timer_stub__E                                 
8000a9fc  xdc_runtime_System_vprintf__E                                           
8000aa38  ti_sysbios_family_arm_a8_Cache_getEnabled__E                            
8000aa70  xdc_runtime_LoggerBuf_reset__E                                          
8000aaa8  ti_sysbios_BIOS_errorRaiseHook__I                                       
8000aadc  ti_sysbios_BIOS_registerRTSLock__I                                      
8000ab10  ti_sysbios_BIOS_removeRTSLock__I                                        
8000ab44  ti_sysbios_BIOS_RtsGateProxy_Object__delete__S                          
8000ab44  ti_sysbios_gates_GateMutex_Object__delete__S                            
8000ab44  ti_sysbios_heaps_HeapMem_Module_GateProxy_Object__delete__S             
8000ab78  ti_sysbios_knl_Clock_Module_startup__E                                  
8000abac  ti_sysbios_knl_Idle_run__E                                              
8000abe0  ti_sysbios_knl_Task_enter__I                                            
8000ac14  xdc_runtime_LoggerBuf_Object__delete__S                                 
8000ac48  xdc_runtime_Registry_findById__E                                        
8000ac7c  xdc_runtime_SysMin_Module_startup__E                                    
8000acb0  ti_sysbios_family_arm_a8_Mmu_enableAsm__I                               
8000ace0  ti_sysbios_BIOS_rtsLock__I                                              
8000ad10  ti_sysbios_gates_GateHwi_Object__delete__S                              
8000ad10  xdc_runtime_LoggerBuf_Module_GateProxy_Object__delete__S                
8000ad10  xdc_runtime_Main_Module_GateProxy_Object__delete__S                     
8000ad10  xdc_runtime_System_Module_GateProxy_Object__delete__S                   
8000ad40  ti_sysbios_gates_GateMutex_Instance_init__E                             
8000ad70  ti_sysbios_heaps_HeapMem_Object__delete__S                              
8000ad70  xdc_runtime_Memory_HeapProxy_Object__delete__S                          
8000ada0  xdc_runtime_Error_raiseX__E                                             
8000add0  xdc_runtime_Memory_valloc__E                                            
8000ae00  xdc_runtime_SysMin_exit__E                                              
8000ae00  xdc_runtime_System_SupportProxy_exit__E                                 
8000ae30  ti_sysbios_gates_GateHwi_Handle__label__S                               
8000ae30  xdc_runtime_LoggerBuf_Module_GateProxy_Handle__label__S                 
8000ae30  xdc_runtime_Main_Module_GateProxy_Handle__label__S                      
8000ae30  xdc_runtime_System_Module_GateProxy_Handle__label__S                    
8000ae5c  ti_sysbios_BIOS_RtsGateProxy_Handle__label__S                           
8000ae5c  ti_sysbios_gates_GateMutex_Handle__label__S                             
8000ae5c  ti_sysbios_heaps_HeapMem_Module_GateProxy_Handle__label__S              
8000ae88  ti_sysbios_gates_GateMutex_leave__E                                     
8000aeb4  ti_sysbios_heaps_HeapMem_Handle__label__S                               
8000aeb4  xdc_runtime_Memory_HeapProxy_Handle__label__S                           
8000aee0  ti_sysbios_knl_Semaphore_Object__destruct__S                            
8000af0c  xdc_runtime_Error_check__E                                              
8000af38  xdc_runtime_LoggerBuf_Handle__label__S                                  
8000af64  ti_sysbios_BIOS_rtsUnlock__I                                            
8000af8c  ti_sysbios_BIOS_startFunc__I                                            
8000afb4  ti_sysbios_family_arm_a8_intcps_Hwi_Module__startupDone__F              
8000afb4  ti_sysbios_family_arm_a8_intcps_Hwi_Module__startupDone__S              
8000afb4  ti_sysbios_hal_Hwi_HwiProxy_Module__startupDone__S                      
8000afdc  ti_sysbios_family_arm_a8_ti81xx_TimerSupport_Module__startupDone__F     
8000afdc  ti_sysbios_family_arm_a8_ti81xx_TimerSupport_Module__startupDone__S     
8000afdc  ti_sysbios_timers_dmtimer_Timer_TimerSupportProxy_Module__startupDone__S
8000b004  ti_sysbios_knl_Queue_Object__destruct__S                                
8000b02c  ti_sysbios_knl_Clock_TimerProxy_Module__startupDone__S                  
8000b02c  ti_sysbios_timers_dmtimer_Timer_Module__startupDone__F                  
8000b02c  ti_sysbios_timers_dmtimer_Timer_Module__startupDone__S                  
8000b054  xdc_runtime_System_abort__E                                             
8000b07c  xdc_runtime_System_aprintf__E                                           
8000b0a4  xdc_runtime_System_printf__E                                            
8000b0cc  _register_unlock                                                        
8000b0d8  _register_lock                                                          
8000b0e4  _nop                                                                    
8000b0f0  ti_sysbios_family_arm_a8_intcps_Hwi_init__I                             
8000b114  ti_sysbios_knl_Task_sleepTimeout__I                                     
8000b138  xdc_runtime_System_exit__E                                              
8000b15c  ti_sysbios_family_arm_a8_Mmu_disableAsm__I                              
8000b17c  _args_main                                                              
8000b19c  ti_sysbios_BIOS_exitFunc__I                                             
8000b1bc  ti_sysbios_family_arm_a8_intcps_Hwi_startup__E                          
8000b1bc  ti_sysbios_hal_Hwi_HwiProxy_startup__E                                  
8000b1dc  xdc_runtime_LoggerBuf_Instance_finalize__E                              
8000b1fc  xdc_runtime_LoggerBuf_write2__E                                         
8000b21c  ti_sysbios_family_arm_TaskSupport_glue                                  
8000b238  strlen                                                                  
8000b254  ti_sysbios_family_arm_a8_Cache_disableBP__E                             
8000b270  ti_sysbios_family_arm_a8_Cache_disableL1d__I                            
8000b28c  ti_sysbios_family_arm_a8_Cache_enableBP__E                              
8000b2a8  ti_sysbios_family_arm_a8_TimestampProvider_initCCNT__I                  
8000b2c4  ti_sysbios_heaps_HeapMem_Object__get__S                                 
8000b2e0  ti_sysbios_knl_Swi_Object__get__S                                       
8000b2fc  xdc_runtime_LoggerBuf_Object__get__S                                    
8000b318  xdc_runtime_LoggerBuf_write0__E                                         
8000b334  xdc_runtime_LoggerBuf_write1__E                                         
8000b350  xdc_runtime_Startup_exec__I                                             
8000b36c  xdc_runtime_SysMin_ready__E                                             
8000b36c  xdc_runtime_System_SupportProxy_ready__E                                
8000b388  xdc_runtime_System_vsnprintf__E                                         
8000b3a4  xdc_runtime_Text_ropeText__E                                            
8000b3c0  ti_sysbios_family_arm_TaskSupport_swap__E                               
8000b3c0  ti_sysbios_knl_Task_SupportProxy_swap__E                                
8000b3d8  strcpy                                                                  
8000b3f0  ti_sysbios_BIOS_exit__E                                                 
8000b408  ti_sysbios_BIOS_setThreadType__E                                        
8000b420  ti_sysbios_BIOS_start__E                                                
8000b438  ti_sysbios_hal_Hwi_Module_startup__E                                    
8000b450  ti_sysbios_knl_Queue_empty__E                                           
8000b468  ti_sysbios_knl_Swi_disable__E                                           
8000b480  ti_sysbios_knl_Task_Object__get__S                                      
8000b498  ti_sysbios_knl_Task_disable__E                                          
8000b4b0  xdc_runtime_Error_init__E                                               
8000b4c8  xdc_runtime_Text_visitRope__I                                           
8000b4e0  ti_sysbios_family_arm_a8_Mmu_init__I                                    
8000b4f4  ti_sysbios_family_arm_a8_Mmu_isEnabled__E                               
8000b508  __TI_decompress_none                                                    
8000b51c  ti_sysbios_family_arm_TaskSupport_checkStack__E                         
8000b51c  ti_sysbios_knl_Task_SupportProxy_checkStack__E                          
8000b530  ti_sysbios_family_arm_a8_Cache_disableL1p__I                            
8000b544  ti_sysbios_family_arm_a8_Cache_enableL1p__I                             
8000b558  ti_sysbios_family_arm_a8_intcps_Hwi_clearInterrupt__E                   
8000b558  ti_sysbios_hal_Hwi_HwiProxy_clearInterrupt__E                           
8000b56c  ti_sysbios_family_arm_a8_intcps_Hwi_switchFromBootStack__E              
8000b56c  ti_sysbios_hal_Hwi_HwiProxy_switchFromBootStack__E                      
8000b580  ti_sysbios_gates_GateMutex_Instance_finalize__E                         
8000b594  ti_sysbios_knl_Semaphore_Instance_finalize__E                           
8000b5a8  xdc_runtime_Gate_leaveSystem__E                                         
8000b5bc  xdc_runtime_Memory_HeapProxy_alloc__E                                   
8000b5d0  xdc_runtime_Memory_HeapProxy_free__E                                    
8000b5e4  xdc_runtime_LoggerBuf_disable__E                                        
8000b5f8  xdc_runtime_LoggerBuf_enable__E                                         
8000b60c  xdc_runtime_Memory_calloc__E                                            
8000b620  xdc_runtime_Memory_free__E                                              
8000b634  __TI_zero_init                                                          
8000b644  ti_sysbios_BIOS_getCpuFreq__E                                           
8000b644  ti_sysbios_family_arm_a8_TimestampProvider_getFreq__E                   
8000b644  xdc_runtime_LoggerBuf_TimestampProxy_getFreq__E                         
8000b644  xdc_runtime_Timestamp_SupportProxy_getFreq__E                           
8000b654  ti_sysbios_family_arm_TaskSupport_getStackAlignment__E                  
8000b654  ti_sysbios_knl_Task_SupportProxy_getStackAlignment__E                   
8000b664  ti_sysbios_family_arm_a8_Cache_disableL2__I                             
8000b674  ti_sysbios_family_arm_a8_Cache_enableL1d__I                             
8000b684  ti_sysbios_family_arm_a8_Cache_enableL2__I                              
8000b694  ti_sysbios_family_arm_a8_TimestampProvider_Module_startup__E            
8000b6a4  ti_sysbios_family_arm_a8_intcps_Hwi_initVbar__I                         
8000b6a4  xdc_runtime_Startup_reset__I                                            
8000b6b4  ti_sysbios_family_arm_exc_Exception_Module_startup__E                   
8000b6c4  ti_sysbios_gates_GateHwi_enter__E                                       
8000b6d4  ti_sysbios_knl_Queue_Object__get__S                                     
8000b6e4  xdc_runtime_Gate_enterSystem__E                                         
8000b6f4  xdc_runtime_Memory_getMaxDefaultTypeAlign__E                            
8000b704  xdc_runtime_Startup_rtsDone__E                                          
8000b714  ti_sysbios_family_arm_a8_Cache_getCacheLevelInfo__I                     
8000b720  ti_sysbios_knl_Idle_loop__E                                             
8000b72c  ti_sysbios_knl_Queue_Instance_init__E                                   
8000b738  ti_sysbios_timers_dmtimer_Timer_getMaxTicks__E                          
8000b744  __xdc__init                                                             
8000b74c  ti_sysbios_family_arm_a8_Mmu_setDomainAccessCtrlReg__E                  
8000b754  __TI_decompress_rle24                                                   
8000b75c  ti_sysbios_family_arm_TaskSupport_Module__startupDone__S                
8000b75c  ti_sysbios_knl_Task_SupportProxy_Module__startupDone__S                 
8000b764  ti_sysbios_family_arm_a8_Cache_getLockdownReg__I                        
8000b76c  ti_sysbios_family_arm_a8_Cache_invL1pAll__E                             
8000b774  ti_sysbios_family_arm_a8_Cache_setLockdownReg__I                        
8000b77c  ti_sysbios_family_arm_a8_TimestampProvider_get32__E                     
8000b77c  xdc_runtime_LoggerBuf_TimestampProxy_get32__E                           
8000b77c  xdc_runtime_Timestamp_SupportProxy_get32__E                             
8000b784  ti_sysbios_family_arm_a8_ti81xx_TimerSupport_Module_startup__E          
8000b78c  ti_sysbios_gates_GateHwi_leave__E                                       
8000b794  ti_sysbios_gates_GateHwi_query__E                                       
8000b794  xdc_runtime_LoggerBuf_Module_GateProxy_query__E                         
8000b794  xdc_runtime_Main_Module_GateProxy_query__E                              
8000b794  xdc_runtime_System_Module_GateProxy_query__E                            
8000b79c  ti_sysbios_BIOS_RtsGateProxy_query__E                                   
8000b79c  ti_sysbios_gates_GateMutex_query__E                                     
8000b79c  ti_sysbios_heaps_HeapMem_Module_GateProxy_query__E                      
8000b7a4  ti_sysbios_heaps_HeapMem_isBlocking__E                                  
8000b7ac  xdc_runtime_Error_getSite__E                                            
8000b7b4  xdc_runtime_System_Module_startup__E                                    
8000b7bc  LoggerBuf_instanceStartup                                               
8000b7c0  ti_sysbios_BIOS_RtsGateProxy_enter__E                                   
8000b7c4  ti_sysbios_BIOS_RtsGateProxy_leave__E                                   
8000b7c8  ti_sysbios_BIOS_nullFunc__I                                             
8000b7cc  ti_sysbios_family_arm_a8_ti81xx_TimerSupport_enable__E                  
8000b7cc  ti_sysbios_timers_dmtimer_Timer_TimerSupportProxy_enable__E             
8000b7d0  ti_sysbios_gates_GateHwi_Instance_init__E                               
8000b7d4  ti_sysbios_heaps_HeapMem_Module_GateProxy_enter__E                      
8000b7d8  ti_sysbios_heaps_HeapMem_Module_GateProxy_leave__E                      
8000b7dc  ti_sysbios_knl_Clock_TimerProxy_getMaxTicks__E                          
8000b7e0  ti_sysbios_knl_Queue_destruct                                           
8000b7e4  ti_sysbios_knl_Semaphore_destruct                                       
8000b7e8  ti_sysbios_knl_Task_startup__E                                          
8000b7ec  xdc_runtime_LoggerBuf_Module_GateProxy_enter__E                         
8000b7f0  xdc_runtime_LoggerBuf_Module_GateProxy_leave__E                         
8000b7f4  xdc_runtime_System_Module_GateProxy_enter__E                            
8000b7f8  xdc_runtime_System_Module_GateProxy_leave__E                            
8000b7fc  xdc_runtime_System_aprintf_va__F                                        
8000b800  xdc_runtime_System_printf_va__F                                         
8000b804  ti_sysbios_family_arm_TaskSupport_stackAlignment__C                     
8000b808  ti_sysbios_family_arm_exc_Exception_Module_State_0_excStack_0__A        
8000d808  ti_sysbios_heaps_HeapMem_Instance_State_0_buf__A                        
8000e808  ti_sysbios_knl_Task_Instance_State_0_stack__A                           
8000f008  ti_sysbios_family_arm_a8_intcps_Hwi_Module_State_0_fiqStack__A          
8000f408  xdc_runtime_LoggerBuf_Instance_State_0_entryArr__A                      
8000f608  xdc_runtime_SysMin_Module_State_0_outbuf__A                             
8000f808  __CIOBUF_                                                               
8000f930  xdc_runtime_Text_nodeTab__A                                             
8000fa58  ti_sysbios_knl_Task_Object__PARAMS__C                                   
8000fa94  xdc_runtime_LoggerBuf_Module__FXNS__C                                   
8000fad0  xdc_runtime_Startup_sfxnTab__A                                          
8000fb04  ti_sysbios_heaps_HeapMem_Module__FXNS__C                                
8000fb2c  ti_sysbios_gates_GateHwi_Module__FXNS__C                                
8000fb50  ti_sysbios_gates_GateMutex_Module__FXNS__C                              
8000fb74  ti_sysbios_heaps_HeapMem_Object__PARAMS__C                              
8000fb98  ti_sysbios_knl_Semaphore_Object__PARAMS__C                              
8000fbbc  xdc_runtime_LoggerBuf_Object__PARAMS__C                                 
8000fbe0  ti_sysbios_gates_GateHwi_Object__DESC__C                                
8000fc00  ti_sysbios_gates_GateMutex_Object__DESC__C                              
8000fc20  ti_sysbios_heaps_HeapMem_Object__DESC__C                                
8000fc40  ti_sysbios_knl_Queue_Object__DESC__C                                    
8000fc60  ti_sysbios_knl_Semaphore_Object__DESC__C                                
8000fc80  ti_sysbios_knl_Task_Object__DESC__C                                     
8000fca0  xdc_runtime_LoggerBuf_Object__DESC__C                                   
8000fcc0  xdc_runtime_Startup_sfxnRts__A                                          
8000fcda  ti_sysbios_family_arm_a8_Cache_branchPredictionEnabled__C               
8000fcdc  ti_sysbios_gates_GateHwi_Object__PARAMS__C                              
8000fcf4  ti_sysbios_gates_GateMutex_Object__PARAMS__C                            
8000fd0c  ti_sysbios_knl_Queue_Object__PARAMS__C                                  
8000fd35  xdc_runtime_Error_policy__C                                             
8000fd36  ti_sysbios_family_arm_a8_Mmu_defaultAttrs__C                            
8000fd46  ti_sysbios_family_arm_a8_Cache_enableCache__C                           
8000fd48  xdc_runtime_Startup_firstFxns__A                                        
8000fd54  ti_sysbios_knl_Idle_funcList__C                                         
8000fd5c  xdc_runtime_Startup_firstFxns__C                                        
8000fd64  xdc_runtime_Startup_lastFxns__C                                         
8000fd6c  ti_sysbios_family_arm_a8_Mmu_A_nullPointer__C                           
8000fd70  ti_sysbios_family_arm_a8_Mmu_A_unknownDescType__C                       
8000fd74  ti_sysbios_family_arm_a8_Mmu_Module__diagsEnabled__C                    
8000fd78  ti_sysbios_family_arm_a8_Mmu_Module__diagsIncluded__C                   
8000fd7c  ti_sysbios_family_arm_a8_Mmu_Module__diagsMask__C                       
8000fd80  ti_sysbios_family_arm_a8_intcps_Hwi_E_undefined__C                      
8000fd84  ti_sysbios_family_arm_a8_intcps_Hwi_LD_end__C                           
8000fd88  ti_sysbios_family_arm_a8_intcps_Hwi_LM_begin__C                         
8000fd8c  ti_sysbios_family_arm_a8_intcps_Hwi_Module__diagsEnabled__C             
8000fd90  ti_sysbios_family_arm_a8_intcps_Hwi_Module__diagsIncluded__C            
8000fd94  ti_sysbios_family_arm_a8_intcps_Hwi_Module__diagsMask__C                
8000fd98  ti_sysbios_family_arm_a8_intcps_Hwi_Module__loggerFxn1__C               
8000fd9c  ti_sysbios_family_arm_a8_intcps_Hwi_Module__loggerFxn8__C               
8000fda0  ti_sysbios_family_arm_a8_intcps_Hwi_Module__loggerObj__C                
8000fda4  ti_sysbios_family_arm_a8_intcps_Hwi_NUM_PRIORITIES__C                   
8000fda8  ti_sysbios_family_arm_a8_intcps_Hwi_taskDisable__C                      
8000fdac  ti_sysbios_family_arm_a8_intcps_Hwi_taskRestoreHwi__C                   
8000fdb0  ti_sysbios_family_arm_exc_Exception_E_dataAbort__C                      
8000fdb4  ti_sysbios_family_arm_exc_Exception_E_prefetchAbort__C                  
8000fdb8  ti_sysbios_family_arm_exc_Exception_E_swi__C                            
8000fdbc  ti_sysbios_family_arm_exc_Exception_E_undefinedInstruction__C           
8000fdc0  ti_sysbios_family_arm_exc_Exception_excHookFuncs__A                     
8000fdc4  ti_sysbios_family_arm_exc_Exception_excHookFuncs__C                     
8000fdc8  ti_sysbios_gates_GateMutex_A_badContext__C                              
8000fdcc  ti_sysbios_gates_GateMutex_Instance_State_sem__O                        
8000fdd0  ti_sysbios_gates_GateMutex_Module__diagsEnabled__C                      
8000fdd4  ti_sysbios_gates_GateMutex_Module__diagsIncluded__C                     
8000fdd8  ti_sysbios_gates_GateMutex_Module__diagsMask__C                         
8000fddc  ti_sysbios_hal_Hwi_E_stackOverflow__C                                   
8000fde0  ti_sysbios_heaps_HeapMem_A_align__C                                     
8000fde4  ti_sysbios_heaps_HeapMem_A_heapSize__C                                  
8000fde8  ti_sysbios_heaps_HeapMem_A_invalidFree__C                               
8000fdec  ti_sysbios_heaps_HeapMem_A_zeroBlock__C                                 
8000fdf0  ti_sysbios_heaps_HeapMem_E_memory__C                                    
8000fdf4  ti_sysbios_heaps_HeapMem_Module__diagsEnabled__C                        
8000fdf8  ti_sysbios_heaps_HeapMem_Module__diagsIncluded__C                       
8000fdfc  ti_sysbios_heaps_HeapMem_Module__diagsMask__C                           
8000fe00  ti_sysbios_heaps_HeapMem_Module__gateObj__C                             
8000fe04  ti_sysbios_heaps_HeapMem_Object__count__C                               
8000fe08  ti_sysbios_heaps_HeapMem_reqAlign__C                                    
8000fe0c  ti_sysbios_knl_Clock_LM_begin__C                                        
8000fe10  ti_sysbios_knl_Clock_LM_tick__C                                         
8000fe14  ti_sysbios_knl_Clock_LW_delayed__C                                      
8000fe18  ti_sysbios_knl_Clock_Module_State_clockQ__O                             
8000fe1c  ti_sysbios_knl_Clock_Module__diagsEnabled__C                            
8000fe20  ti_sysbios_knl_Clock_Module__diagsIncluded__C                           
8000fe24  ti_sysbios_knl_Clock_Module__diagsMask__C                               
8000fe28  ti_sysbios_knl_Clock_Module__loggerFxn1__C                              
8000fe2c  ti_sysbios_knl_Clock_Module__loggerFxn2__C                              
8000fe30  ti_sysbios_knl_Clock_Module__loggerObj__C                               
8000fe34  ti_sysbios_knl_Idle_funcList__A                                         
8000fe38  ti_sysbios_knl_Semaphore_A_badContext__C                                
8000fe3c  ti_sysbios_knl_Semaphore_A_noEvents__C                                  
8000fe40  ti_sysbios_knl_Semaphore_A_overflow__C                                  
8000fe44  ti_sysbios_knl_Semaphore_A_pendTaskDisabled__C                          
8000fe48  ti_sysbios_knl_Semaphore_Instance_State_pendQ__O                        
8000fe4c  ti_sysbios_knl_Semaphore_LM_pend__C                                     
8000fe50  ti_sysbios_knl_Semaphore_LM_post__C                                     
8000fe54  ti_sysbios_knl_Semaphore_Module__diagsEnabled__C                        
8000fe58  ti_sysbios_knl_Semaphore_Module__diagsIncluded__C                       
8000fe5c  ti_sysbios_knl_Semaphore_Module__diagsMask__C                           
8000fe60  ti_sysbios_knl_Semaphore_Module__loggerFxn2__C                          
8000fe64  ti_sysbios_knl_Semaphore_Module__loggerFxn4__C                          
8000fe68  ti_sysbios_knl_Semaphore_Module__loggerObj__C                           
8000fe6c  ti_sysbios_knl_Swi_LD_end__C                                            
8000fe70  ti_sysbios_knl_Swi_LM_begin__C                                          
8000fe74  ti_sysbios_knl_Swi_LM_post__C                                           
8000fe78  ti_sysbios_knl_Swi_Module__diagsEnabled__C                              
8000fe7c  ti_sysbios_knl_Swi_Module__diagsIncluded__C                             
8000fe80  ti_sysbios_knl_Swi_Module__diagsMask__C                                 
8000fe84  ti_sysbios_knl_Swi_Module__loggerFxn1__C                                
8000fe88  ti_sysbios_knl_Swi_Module__loggerFxn4__C                                
8000fe8c  ti_sysbios_knl_Swi_Module__loggerObj__C                                 
8000fe90  ti_sysbios_knl_Swi_Object__count__C                                     
8000fe94  ti_sysbios_knl_Task_A_badPriority__C                                    
8000fe98  ti_sysbios_knl_Task_A_badTaskState__C                                   
8000fe9c  ti_sysbios_knl_Task_A_badThreadType__C                                  
8000fea0  ti_sysbios_knl_Task_A_badTimeout__C                                     
8000fea4  ti_sysbios_knl_Task_A_noPendElem__C                                     
8000fea8  ti_sysbios_knl_Task_A_sleepTaskDisabled__C                              
8000feac  ti_sysbios_knl_Task_E_spOutOfBounds__C                                  
8000feb0  ti_sysbios_knl_Task_E_stackOverflow__C                                  
8000feb4  ti_sysbios_knl_Task_LD_block__C                                         
8000feb8  ti_sysbios_knl_Task_LD_exit__C                                          
8000febc  ti_sysbios_knl_Task_LD_ready__C                                         
8000fec0  ti_sysbios_knl_Task_LM_sleep__C                                         
8000fec4  ti_sysbios_knl_Task_LM_switch__C                                        
8000fec8  ti_sysbios_knl_Task_Module_State_inactiveQ__O                           
8000fecc  ti_sysbios_knl_Task_Module__diagsEnabled__C                             
8000fed0  ti_sysbios_knl_Task_Module__diagsIncluded__C                            
8000fed4  ti_sysbios_knl_Task_Module__diagsMask__C                                
8000fed8  ti_sysbios_knl_Task_Module__loggerFxn2__C                               
8000fedc  ti_sysbios_knl_Task_Module__loggerFxn4__C                               
8000fee0  ti_sysbios_knl_Task_Module__loggerObj__C                                
8000fee4  ti_sysbios_knl_Task_Object__count__C                                    
8000fee8  ti_sysbios_knl_Task_allBlockedFunc__C                                   
8000feec  ti_sysbios_knl_Task_defaultStackHeap__C                                 
8000fef0  ti_sysbios_knl_Task_defaultStackSize__C                                 
8000fef4  ti_sysbios_knl_Task_numConstructedTasks__C                              
8000fef8  ti_sysbios_timers_dmtimer_Timer_E_cannotSupport__C                      
8000fefc  ti_sysbios_timers_dmtimer_Timer_E_freqMismatch__C                       
8000ff00  ti_sysbios_timers_dmtimer_Timer_Module__diagsEnabled__C                 
8000ff04  ti_sysbios_timers_dmtimer_Timer_Module__diagsIncluded__C                
8000ff08  ti_sysbios_timers_dmtimer_Timer_Module__diagsMask__C                    
8000ff0c  ti_sysbios_timers_dmtimer_Timer_numTimerDevices__C                      
8000ff10  xdc_runtime_Assert_E_assertFailed__C                                    
8000ff14  xdc_runtime_Core_A_initializedParams__C                                 
8000ff18  xdc_runtime_Core_Module__diagsEnabled__C                                
8000ff1c  xdc_runtime_Core_Module__diagsIncluded__C                               
8000ff20  xdc_runtime_Core_Module__diagsMask__C                                   
8000ff24  xdc_runtime_Error_E_memory__C                                           
8000ff28  xdc_runtime_Error_Module__diagsEnabled__C                               
8000ff2c  xdc_runtime_Error_Module__diagsIncluded__C                              
8000ff30  xdc_runtime_Error_Module__diagsMask__C                                  
8000ff34  xdc_runtime_Error_Module__loggerFxn8__C                                 
8000ff38  xdc_runtime_Error_Module__loggerObj__C                                  
8000ff3c  xdc_runtime_Error_policyFxn__C                                          
8000ff40  xdc_runtime_Error_raiseHook__C                                          
8000ff44  xdc_runtime_IFilterLogger_Interface__BASE__C                            
8000ff48  xdc_runtime_IGateProvider_Interface__BASE__C                            
8000ff4c  xdc_runtime_IHeap_Interface__BASE__C                                    
8000ff50  xdc_runtime_ILogger_Interface__BASE__C                                  
8000ff54  xdc_runtime_IModule_Interface__BASE__C                                  
8000ff58  xdc_runtime_Log_L_error__C                                              
8000ff5c  xdc_runtime_LoggerBuf_E_badLevel__C                                     
8000ff60  xdc_runtime_LoggerBuf_Module__gateObj__C                                
8000ff64  xdc_runtime_LoggerBuf_Object__count__C                                  
8000ff68  xdc_runtime_LoggerBuf_statusLogger__C                                   
8000ff6c  xdc_runtime_Memory_defaultHeapInstance__C                               
8000ff70  xdc_runtime_Startup_execImpl__C                                         
8000ff74  xdc_runtime_Startup_maxPasses__C                                        
8000ff78  xdc_runtime_Startup_sfxnRts__C                                          
8000ff7c  xdc_runtime_Startup_sfxnTab__C                                          
8000ff80  xdc_runtime_SysMin_bufSize__C                                           
8000ff84  xdc_runtime_SysMin_outputFunc__C                                        
8000ff88  xdc_runtime_System_Module__gateObj__C                                   
8000ff8c  xdc_runtime_System_abortFxn__C                                          
8000ff90  xdc_runtime_System_exitFxn__C                                           
8000ff94  xdc_runtime_System_extendFxn__C                                         
8000ff98  xdc_runtime_System_maxAtexitHandlers__C                                 
8000ff9c  xdc_runtime_Text_charTab__C                                             
8000ffa0  xdc_runtime_Text_nameEmpty__C                                           
8000ffa4  xdc_runtime_Text_nameStatic__C                                          
8000ffa8  xdc_runtime_Text_nameUnknown__C                                         
8000ffac  xdc_runtime_Text_nodeTab__C                                             
8000ffb0  xdc_runtime_Text_visitRopeFxn__C                                        
8000ffb4  ti_sysbios_family_arm_a8_Cache_unlockL2Cache__C                         
8000ffb6  ti_sysbios_family_arm_a8_Mmu_Module__id__C                              
8000ffb8  ti_sysbios_family_arm_a8_Mmu_enableMMU__C                               
8000ffba  ti_sysbios_family_arm_a8_intcps_Hwi_Module__id__C                       
8000ffbc  ti_sysbios_family_arm_a8_intcps_Hwi_Module__loggerDefined__C            
8000ffbe  ti_sysbios_family_arm_exc_Exception_Module__id__C                       
8000ffc0  ti_sysbios_gates_GateMutex_Module__id__C                                
8000ffc2  ti_sysbios_hal_Hwi_Module__id__C                                        
8000ffc4  ti_sysbios_heaps_HeapMem_Module__id__C                                  
8000ffc6  ti_sysbios_knl_Clock_Module__id__C                                      
8000ffc8  ti_sysbios_knl_Clock_Module__loggerDefined__C                           
8000ffca  ti_sysbios_knl_Semaphore_Module__id__C                                  
8000ffcc  ti_sysbios_knl_Semaphore_Module__loggerDefined__C                       
8000ffce  ti_sysbios_knl_Swi_Module__id__C                                        
8000ffd0  ti_sysbios_knl_Swi_Module__loggerDefined__C                             
8000ffd2  ti_sysbios_knl_Task_Module__id__C                                       
8000ffd4  ti_sysbios_knl_Task_Module__loggerDefined__C                            
8000ffd6  ti_sysbios_knl_Task_initStackFlag__C                                    
8000ffd8  ti_sysbios_timers_dmtimer_Timer_Module__id__C                           
8000ffda  ti_sysbios_timers_dmtimer_Timer_checkFrequency__C                       
8000ffdc  ti_sysbios_timers_dmtimer_Timer_startupNeeded__C                        
8000ffde  xdc_runtime_Core_Module__id__C                                          
8000ffe0  xdc_runtime_Error_Module__loggerDefined__C                              
8000ffe2  xdc_runtime_Error_maxDepth__C                                           
8000ffe4  xdc_runtime_LoggerBuf_Module__id__C                                     
8000ffe6  xdc_runtime_LoggerBuf_filterByLevel__C                                  
8000ffe8  xdc_runtime_Memory_Module__id__C                                        
8000ffea  xdc_runtime_SysMin_flushAtExit__C                                       
8000ffec  xdc_runtime_Text_charCnt__C                                             
8000ffee  xdc_runtime_Text_isLoaded__C                                            
8000fff0  xdc_runtime_Text_registryModsLastId__C                                  
8000fff2  xdc_runtime_Text_unnamedModsLastId__C                                   
8000fff4  _lock                                                                   
8000fff8  _unlock                                                                 
8000fffc  main_func_sp                                                            
80010000  ti_sysbios_family_arm_a8_Mmu_Module_State_0_tableBuf__A                 
80014000  xdc_runtime_Text_charTab__A                                             
80015950  __stack                                                                 
80017950  __STACK_END                                                             
80017950  ti_sysbios_family_arm_a8_intcps_Hwi_Module__state__V                    
80017ba0  ti_sysbios_family_arm_a8_Mmu_Module__state__V                           
80017ba4  ti_sysbios_family_arm_a8_TimestampProvider_Module__state__V             
80017bac  ti_sysbios_family_arm_a8_intcps_Hwi_Module__root__V                     
80017bb4  ti_sysbios_family_arm_a8_intcps_Hwi_Object__table__V                    
80017bd0  ti_sysbios_family_arm_a8_ti81xx_TimerSupport_Module_State_0_intNums__A  
80017bd8  ti_sysbios_family_arm_a8_ti81xx_TimerSupport_Module__state__V           
80017bdc  ti_sysbios_family_arm_exc_Exception_Module_State_0_excActive__A         
80017be0  ti_sysbios_family_arm_exc_Exception_Module_State_0_excContext__A        
80017be4  ti_sysbios_family_arm_exc_Exception_Module_State_0_excStackBuffers__A   
80017be8  ti_sysbios_family_arm_exc_Exception_Module_State_0_excStack__A          
80017bec  ti_sysbios_family_arm_exc_Exception_Module__state__V                    
80017c00  ti_sysbios_gates_GateHwi_Module__root__V                                
80017c08  ti_sysbios_gates_GateHwi_Object__table__V                               
80017c0c  ti_sysbios_gates_GateMutex_Module__root__V                              
80017c14  ti_sysbios_hal_Hwi_Module__root__V                                      
80017c1c  ti_sysbios_hal_Hwi_Object__table__V                                     
80017c24  ti_sysbios_heaps_HeapMem_Module__root__V                                
80017c2c  ti_sysbios_heaps_HeapMem_Object__table__V                               
80017c44  ti_sysbios_knl_Clock_Module__root__V                                    
80017c4c  ti_sysbios_knl_Clock_Object__table__V                                   
80017c6c  ti_sysbios_knl_Queue_Module__root__V                                    
80017c74  ti_sysbios_knl_Semaphore_Module__root__V                                
80017c7c  ti_sysbios_knl_Swi_Module__root__V                                      
80017c84  ti_sysbios_knl_Swi_Module__state__V                                     
80017ca0  ti_sysbios_knl_Task_Module__root__V                                     
80017ca8  ti_sysbios_knl_Task_Module_State_0_idleTask__A                          
80017cac  ti_sysbios_timers_dmtimer_Timer_Module__root__V                         
80017cb4  ti_sysbios_timers_dmtimer_Timer_Module_State_0_handles__A               
80017ccc  ti_sysbios_timers_dmtimer_Timer_Module__state__V                        
80017ce0  xdc_runtime_Error_Module__state__V                                      
80017ce4  xdc_runtime_LoggerBuf_Module__root__V                                   
80017cec  xdc_runtime_LoggerBuf_Module__state__V                                  
80017cf4  xdc_runtime_Memory_Module__state__V                                     
80017cf8  xdc_runtime_Registry_Module__state__V                                   
80017d00  xdc_runtime_Startup_Module__state__V                                    
80017d08  xdc_runtime_SysMin_Module__state__V                                     
80017d14  xdc_runtime_System_Module_State_0_atexitHandlers__A                     
80017d24  xdc_runtime_System_Module__state__V                                     
80017d2c  xdc_runtime_Text_Module__state__V                                       
80017d34  __xdc__init__addr                                                       
80017d38  GpmcMux                                                                 
80017eb8  ti_sysbios_knl_Swi_Module_State_0_readyQ__A                             
80017f38  ti_sysbios_knl_Task_Module_State_0_readyQ__A                            
80017fb8  ti_sysbios_timers_dmtimer_Timer_Object__table__V                        
80018014  applMmuEntries                                                          
8001806c  TSK_idle                                                                
8001806c  ti_sysbios_knl_Task_Object__table__V                                    
800180b8  ti_sysbios_timers_dmtimer_Timer_Module_State_0_device__A                
80018100  ti_sysbios_knl_Task_Module__state__V                                    
80018144  ti_sysbios_gates_GateMutex_Object__table__V                             
8001817c  ti_sysbios_family_arm_a8_Cache_Module__state__V                         
800181b0  ti_sysbios_knl_Swi_Object__table__V                                     
800181e0  ti_sysbios_timers_dmtimer_Timer_Module_State_0_intFreqs__A              
80018210  ti_sysbios_knl_Clock_Module__state__V                                   
8001823c  ti_sysbios_BIOS_Module__state__V                                        
80018260  xdc_runtime_LoggerBuf_Object__table__V                                  
80018284  __TI_cleanup_ptr                                                        
80018288  __TI_dtors_ptr                                                          
80018400  ti_sysbios_family_arm_a8_intcps_Hwi_vectors                             
80018440  __TI_static_base__                                                      
80018b3c  __TI_Handler_Table_Base                                                 
80018b48  __TI_Handler_Table_Limit                                                
80018b50  __TI_CINIT_Base                                                         
80018b68  __TI_CINIT_Limit                                                        
ffffffff  __binit__                                                               
ffffffff  __c_args__                                                              
ffffffff  binit                                                                   
UNDEFED   SHT$$INIT_ARRAY$$Base                                                   
UNDEFED   SHT$$INIT_ARRAY$$Limit                                                  

[754 symbols]
